:020000041100E9
:10300000002370B5284C0120636101F029FA4020AB
:103010000223FE21254A207401F0A8FA002833D1AA
:103020000223FF21224A207C01F0A0FA00282BD1A4
:10303000204BA2899A4224D1E3891F4A93420CD1A2
:103040001E4B63611E4B2268002A03D1002B01D066
:1030500023CB23C401F078FA70BD1A4A934201D001
:103060000023F0E7184B194A1B68934205D9C02288
:103070000421207C920001F0F3FA104B6361144BA1
:10308000E1E700232374EBE7CC223820AC21920146
:10309000207401F0E5FA0028F3D10E4B63610E4B6A
:1030A000E3810E4BCFE7C0468863FF1F9463FF1F89
:1030B0009663FF1F5959000083050000C1420011AB
:1030C0004CBE001182150000AC63FF1F8713000087
:1030D00058BE00115D430011AAAAFFFF40BE0011B7
:1030E000F7B5164B0192C318021D002000938823E8
:1030F0005B05D3181B685C1C1AD09CB2402C18D8F6
:103100008D781E0CAC466746CD782D023D43AE420D
:1031100006D1019800280ED110000C70240A4C70C2
:1031200003249BB20733A343D218009B9A42DED3F9
:10313000FEBD4432F9E71000FAE7C046FC0F00007C
:10314000802213B503000324019189B25201073193
:103150009B18A14304305A1A88235B05C3181B68C7
:10316000591C03D190429241104016BD99B240299A
:1031700007D80B000733A343C0189042ECD30020BC
:10318000F3E74430F9E7134B134A1B68126810B594
:10319000FA24934201D81A00F824104BE4021B6869
:1031A0009A4210D813000E4A12689A420ED3013385
:1031B00007D1F823DB029C4203D10A49054808F0F5
:1031C00043FC200010BDFC24E402ECE7FE24E402F2
:1031D000F7E7C04600C0071100D0071100E0071153
:1031E00000F00711FFFFFF7FF0B59BB015000490C2
:1031F0000391402A00D9A0E006AB59801A80FFF75E
:10320000C2FF0400042816D9002206A9FFF768FFB0
:10321000052810D906AB1B88AB420CD1002D07D076
:10322000514B2A000499C01808F06EFA002802D108
:1032300001201BB0F0BD06AB1D8020000699FFF7F2
:103240007FFF041E7BD1069B0793FFF79CFF802323
:103250005B01C618802307001B039E4201D3F8269A
:10326000F60288235B05F31801931B68013302D033
:10327000019808F039FB3D49019808F0E5FB3B1D3A
:103280000293331D05938822029B52059B181B68ED
:1032900008935A1C3CD044219AB20091402A04D889
:1032A0000320D11D814389B2009103991B0C8B42ED
:1032B00024D0402A22D80122300008A9FFF710FFAD
:1032C000021E1BD1380008A9FFF70AFF04000428DA
:1032D00031D9009A059B9B1880225201B218934263
:1032E00040D288235B05C118009A09A808F05CFA4F
:1032F0001D4B009A09A9F01808F01EFB009A029BCA
:103300009446634402931A4B029AFB189A42BAD32A
:1033100088235B05FC1821680198013908F094FBAB
:10332000200008F0E1FA039A07AB5A8030000799B1
:10333000FFF706FF0400002C03D1002079E70428E2
:10334000FBD988235B05E018069908F07DFB032371
:10335000EA1C9A4300D16BE7034B0499E01808F08C
:10336000EBFA65E70424ECE704000011FFFFFF7FA0
:10337000F80F0000F7B505001400402A21D80027F7
:1033800001AE71803780FFF7FEFE042816D93A009F
:103390003100FFF7A5FE042810D93688BC420BD0B7
:1033A000BD4209D0221CB44200D9321C064B92B255
:1033B000C118280008F0F8F930B2FEBDC04300B2D1
:1033C000FBE703204042F8E70400001137B5042270
:1033D00004000D0001A81649FFF7CCFF02000428E5
:1033E0000BD1019BA34208D3AB4204D0104901A8E2
:1033F0000195FFF7F9FE01203EBD0E4C2368200029
:10340000019308F071FA019920000139019108F047
:103410001BFB80235B01E418074B9C42EED1042286
:10342000034901A80195FFF7DFFE0020E4E7C0464D
:103430005555000000C007110000081130B589B0D3
:1034400008F08AFC10226946254808F0E5FB254B68
:10345000009A9A420ED1019B029A0F2B33D8002179
:1034600001240698013B08D2002900D00292029B59
:10347000013331D10023029325E0551CF2D1020023
:103480002100EFE710341022200004A908F0C4FB4B
:10349000029B013301D1069B0293882304995B05AB
:1034A000C918059B06981A03120B049105928142D4
:1034B00003D02B4201D108F077F9019B013B019326
:1034C000019B002BDED1029B002B03D004930498B8
:1034D0004168084709B030BDE025014C2D03EFE7F6
:1034E0000000011150485936F7B50F490F4B0A68D3
:1034F00004001A4084235B0013430B60030003277E
:103500001033019300252E00112008F0DDFB084B3D
:103510001B683B40AB4002351E43202DF4D1019B7C
:1035200040C4A342EED1F7BD5CF0004000FEFEFFB8
:1035300064F00040802270B5AD4CAE4BD20000214B
:1035400020001C6008F0D8FB2300AB4A88331A60C7
:10355000AA4B1A786E23002A00D01133E3620A23A3
:103560002365A74B1878A74BA0630138E361C3B26A
:10357000032B01D810232362A34B37226361C82396
:10358000DB00A36123008C331A60082336210F3A35
:10359000E518E16323646264E9670439251DE9677E
:1035A00025003B26BC352E602500C0352B6025004C
:1035B000C4352A6025000636CC352E602500083E2D
:1035C000C8352E602500D03529602100D4310B602C
:1035D0002100D8310A6021000225E0310D6025006C
:1035E0004221DC35296025001B3EE4352E60250094
:1035F000E8352B602500EC352A6022000525F432E1
:1036000015602200F03211602200183190321160F2
:1036100022009432136023003C2298331A60AF23B7
:10362000DB002360794B2363032805D808F034FAC4
:10363000330235371523636096232100FA225B009D
:10364000A360E360C8332361714BFC319200A36433
:103650000A6062626F4A704DA2627322E2656D3A3F
:103660006265A2650232E5644A60022161669621C4
:103670008900A166626709210022E166A2676749A5
:10368000674A684E2167E2673560032811D808F061
:1036900003FA96089EA61023CDE70E23CBE70C2352
:1036A000C9E720001A259C30056020000735A030AE
:1036B00005602000A83003602300FA20F833800062
:1036C000186023006420A433186023005F38AC33F3
:1036D000186023000338B03318602300C630B433B9
:1036E000186023000020B833186023003825FC330D
:1036F0009D604D4D5A665D644C4D9A64DD61962522
:10370000AD001D624A4D9A675D62F53DFF3D9D62C9
:103710001E25484ADD6618675867D9651966DA6755
:10372000BE23C021444A5B00E250444B4900635031
:1037300004316250C4225200A350FA23E4205B00FB
:103740000432A3500432A3503D493E4A3E4BD1605F
:103750003E49800019503E49E938FF3819503D492B
:10376000043019503C491038D1613C4911633C493F
:1037700051633C4911603C49195019003B48F831EC
:1037800008603B49D16582213A4A89005A501A00A3
:1037900039490832D1671A003849B432116088219A
:1037A000374A89005A501A00364988321160364A21
:1037B000DA6408F0B1F8012008F0EEF970BD2000DD
:1037C00014259C30056020000435A03070E72000EF
:1037D00010259C30056020000335A03068E72000EC
:1037E0000E259C30056020000235A03060E7C04601
:1037F0000004FF1F6466FF1F5071FF1F1C46FF1F60
:103800004A0AFF1F3A07000080C3C9019A0200005C
:1038100050C300006A180000280A0000204E000073
:1038200088130000F009FF1F00400011681000001D
:10383000C4090000DC05000040420F001027000012
:10384000FD1BFF1FFC00FF1F0000FF1F252FFF1F98
:103850004D32FF1FE530FF1FD91FFF1FF51FFF1F50
:10386000A121FF1F491FFF1FC528FF1F8D2CFF1F10
:10387000D918FF1FD127FF1F3925FF1F4525FF1F1F
:10388000491EFF1F011FFF1FC11DFF1FF7B50B0CB6
:10389000FF270122009300233C001E001D009446D8
:1038A000019089B262469A401000084018413618CB
:1038B000B6B2FF2F02D1012E00D19FB20098024074
:1038C0001A41AD18ADB2FF2C02D1012D00D19CB22E
:1038D0000133102BE6D10320012E07D1012D04D195
:1038E000019B2401E4191C700138FEBD102EFCD18F
:1038F0000238102DF9D00230F7E710B5064C2378C6
:10390000002B07D10548FFF7EFFD0548FFF7ECFD59
:103910000123237010BDC0462466FF1F3866FF1FB9
:103920002866FF1FF0B58BB00D0001230190102910
:1039300036D8FFF7E2FF00231A001B48C15C0133B1
:103940005218102BFAD1023B002A29D0174B184CE1
:103950001F68002306A9E25C1600FA5C56405E541C
:103960000133102BF7D102AA08F076F82A0002A939
:10397000019808F0E9F908F017F823681B1823608C
:1039800008F012F863681B18636008F00DF8A3686C
:103990001B18A36008F008F8E3681B18E360002315
:1039A00018000BB0F0BDC0463866FF1FBC44FF1FB7
:1039B0002866FF1FF0B50223012400275A4E5B4DF5
:1039C0005B4A33702C7013685A49DBB28B708FB02E
:1039D0001760552B10D0082006F032FCB8420BD0EF
:1039E0003B0021000420544A009708F095F98023F9
:1039F000DB059C62FFF722FD002006F0B9FE07F010
:103A0000ABFEFFF797FD07F0D7FE1F220124002130
:103A10004A4B0EAF1A704A4B1C704A4B19704A4BF6
:103A200019689143163A0A431A6060221968914353
:103A3000403A0A431A6007F067FF07F0EDFEC12025
:103A4000FF21424B80001A588A431A50C522920027
:103A500098588843BF390143995098583C490840C9
:103A60008021C9010143802099509958C00509025D
:103A7000090A0143995080213648490107F0C4FFE3
:103A800003232200344901940093344808F03CF8A1
:103A90002C22334903A807F087FE03AC6178207815
:103AA000023406F0F3FBBC42F8D10121002006F0FD
:103AB00007FD2C4B2C4A196803201140A022D2028A
:103AC0000A431A608022196892040A431A6019682E
:103AD000264A1140802292030A431A60244B254A49
:103AE000934200D8012008F017F807F0E5FE07F030
:103AF000C3FE307807F040FF2878C0B208F07CF8A9
:103B000007F022FE0C49042008F00EF806F0FCFD38
:103B100000F0A4F800F0FEFD00F082FE00F00EFAC6
:103B200000200FB0F0BDC0464A0AFF1F1C46FF1F11
:103B300034F00040B863FF1F3B000108480AFF1F34
:103B4000490AFF1F680AFF1FBCF0004000E100E0C7
:103B5000FF00FFFF2046FF1FA458FF1F2056FF1F36
:103B600068BD001114F00040FF7FF8FFFFFF9FFFCA
:103B70005071FF1F0080FF1F70B500252849294A9A
:103B800029484D6308CA1B051B0DED188242F9D167
:103B90000022264B8B63264B08211A628022254B7C
:103BA0009205DA67244BDA688A43DA60234A12788E
:103BB000012A03D09A6822490A409A600121EE2422
:103BC0002048E40002686C438A430260DA681120EE
:103BD0008A43DA6007F070FF112007F08DFF112093
:103BE00007F002FF184A200C0400642390420AD810
:103BF000FA220023D200904205D9144B0A21C018A2
:103C000007F07AFDC3B2124A1372124BD4801B78AC
:103C1000002B04D1104B1021187808F085F870BDE6
:103C2000000005408805054000060540FF01000032
:103C300000F0004004E100E03CF000404A0AFF1FB1
:103C4000FFDFFFFF00380040B70B000030F8FFFF38
:103C5000A063FF1FDC65FF1FD863FF1F002210B5A4
:103C60001100112008F068F810BD0000F8B500231D
:103C700001250826394F3A4C3B62E3681120AB43DB
:103C8000E360E368B343E36007F036FF112007F019
:103C900013FF112007F0B0FE4023226829001343D0
:103CA000236080236268DB02134380226360A36881
:103CB00007201343A360A3682A4A1340A36080230C
:103CC000A2689B0113431022A360236C93432364D7
:103CD000236C2B43236480235B003B62226B224BCB
:103CE0001A402263626B1A406263A26B1A40A2639D
:103CF000E26B1340E3631D4AE3681340E36006F0A0
:103D0000AFFB2900072006F0DBFB8021184A1120B9
:103D1000536C0B43536407F03FFDFD21154B164ACE
:103D200089005A508023C720626B5B03134363638F
:103D3000E36880003343E360E368104A1D43104B9F
:103D4000E56019581140802212020A431A5080225D
:103D500092051A600B4B5E63F8BDC04600F0004050
:103D60003CF00040FFFFDFFFEFFFEFFFFFFF7FFFB3
:103D7000003800400000FF1F793B0011FF00FFFFEB
:103D800000E100E00000054030B503A804880B20E6
:103D9000002C0ED14968074D087849780902014383
:103DA0000A20A94205D1012120001980024B1B7A6B
:103DB000137030BD192A0000A063FF1FF7B515006E
:103DC00008AA16884A680F4F1478527812022243C4
:103DD0000A24BA4214D10122DBB2019200962A00D1
:103DE00007F0E2FB041E0BD1074B1B68002B07D02A
:103DF00068782A78000210434242504101309847C7
:103E00002000FEBD022900002463FF1F30B50125FC
:103E100003790400BFB02B4212D00A49408806F053
:103E20002FFF28420CD06A46074B69465B8D5580B0
:103E30001380064B60881B7A1371002203F0E6FFA3
:103E40003FB030BD1C63FF1F6042FF1FA063FF1F18
:103E500010B50549054806F0C9FE0421044A054885
:103E600006F086FE10BDC0461C63FF1FFFFF00006A
:103E700094BD00116042FF1F10B5024804F048FED7
:103E800010BDC0460D3E0011062310B583701033DF
:103E90000371443B43712A3383714433C37100235C
:103EA0000222012103720E4B027041701C88817244
:103EB0004472197A0273C1729A784273DA78827303
:103EC0000322C2731A7902745A7942740C228274E2
:103ED0009A79C274DB7903751123C370152010BD64
:103EE000A063FF1F10B5142007F08EFC124B1422A4
:103EF0000021186007F000FF002007F09DFC012062
:103F000007F0AAFC022007F027FE032004F0A4F823
:103F1000042006F0B9F8052003F0E2FA062003F0C9
:103F2000AFFF072001F07EF9082006F001FE09200E
:103F300000F062FF10BDC0462863FF1F10B507F0F8
:103F400003FD012007F040FC07F0B6FB002010BD88
:103F5000094B10B50400984205D0012904D1200076
:103F6000064906F043FE10BD0229FCD1013904F0D8
:103F70008DFD0028F3D0F6E7FEFF00004E63FF1F23
:103F800030B5012503790400BFB02B4218D00D498C
:103F9000408806F075FE284212D06A460A4B0B494B
:103FA0001B8813800A235380293313716B4609221F
:103FB000581D07F0F9FB00226946608803F026FFD0
:103FC0003FB030BD4E63FF1FFE42FF1FA063FF1FC7
:103FD00070B50D7A100004AA2C0016881022144027
:103FE000154220D1002E20D10A78022A18D14A6821
:103FF000517815780E4A09022943914205D00D4A9D
:10400000914209D01C800A2404E014220A491A8033
:1040100007F0CAFB200070BD0C2208491A80F7E7A0
:104020001C800124F6E70824F4E70B24F2E7C046DD
:10403000F3FF0000F4FF0000A044FF1F70BE00115A
:1040400010B504000749084806F0D0FD074804F001
:104050009FFC0020E40704D50721054A054806F027
:1040600087FD10BD4E63FF1FFFFF0000513F001191
:10407000D8BD0011A442FF1F00B50C4BBFB01A7889
:104080000B4901A800F0FEFB6B4680B25880002867
:1040900009D06A46074B69461B881380064B0022ED
:1040A000188803F0B3FE3FB000BDC0462C63FF1F6D
:1040B0002D63FF1FFE42FF1FFE43FF1F00B50C4B89
:1040C000BFB01A780B4901A801F0E6FD6B4680B23B
:1040D0005880002809D06A46074B69465B8D1380DB
:1040E000064B0022188803F091FE3FB000BDC04689
:1040F0005663FF1F5763FF1FA442FF1FFE43FF1FAE
:10410000F7B50E00377A1C0008AB11003D001A8885
:1041100020231D401F423CD13378022B3BD17368D2
:104120001F785B781B023B431E4FBB4208D01E4FDB
:10413000BB4214D01D4DAB4221D00A252800FEBD44
:10414000002A2AD1142C2AD82200F06807F02CFB70
:10415000174B1C70012CF1D9FFF7B0FFEEE7002AD6
:104160001BD1202C1BD82200F06807F01DFB114B3F
:1041700004211C70104B187807F0D6FDDEE7E3B27F
:104180000124009201940A00310007F00DFA0500A5
:10419000D4E70825D2E70125D0E70B25CEE70D258A
:1041A000CCE7C046F3FF0000F4FF00000229000046
:1041B0005663FF1F2C63FF1FD863FF1F10B5024813
:1041C00004F0A6FC10BDC046813F001170B516007A
:1041D00004AA148805AA15784A6850781178000254
:1041E0002A4A0843801805284BD807F055FC0313CA
:1041F0001E29343F0720032C0BD80422121BAA428D
:1042000000D92A0022491A803000091907F0CCFA97
:10421000002070BD0720112CFBD81222121BAA42CD
:1042200000D92A001B491A80EEE707200E2CF0D88F
:104230000F22121BAA4200D92A0017491A80E3E76D
:104240000720032CE5D80422121BAA4200D92A0019
:1042500012491A80D8E70720032CDAD80422121B4F
:10426000AA4200D92A000E491A80CDE70720032C64
:10427000CFD80422121BAA4200D92A0009491A8069
:10428000C2E700220A201A80C3E7C046DCD5FFFF40
:1042900023BE00117463FF1F13BE00110EBE001178
:1042A00009BE001104BE001110B50D21024A0348D9
:1042B00006F05EFC10BDC046F8BD00111443FF1FA0
:1042C00037B5002000F0CCF8204D214BEA89287C3E
:1042D0009A422AD1042201A900F076F9040000F0E4
:1042E00033F9002C30D16B4699882B68C9BA4B43FF
:1042F0002989184A1B145B1853806B46D9886B6850
:1043000049BA89B24B4369891B0C5B181248191CC6
:104310001BB2834200DD011C0B0400D50021138871
:1043200091800133138020003EBD0223002101AAA9
:1043300000F01CF96A46040002230121287C0632A1
:1043400000F014F90443CAE70124ECE78863FF1F77
:1043500083050000A063FF1F0F27000037B5012071
:1043600000F07EF81F4D07226946287C00F02CF9EA
:10437000041E33D16B461B787F2B2FD800F0E4F856
:104380006B46D878F02302041B031A406B469B88C7
:1043900015495BBA9BB21A432B68000953432A891B
:1043A0001B0C9B184B806B465A789B7812031B01A1
:1043B0001A436B68024353436A891B0C9B180B48D2
:1043C0001A1C1BB2834200DD021C130400D500221C
:1043D0000B888A8001330B8020003EBD00F0B4F8CA
:1043E0000124F9E78863FF1FA063FF1F0F27000068
:1043F00010B50F4C237C002B0CD0382B0BD1012097
:1044000000F02EF8CC22AC21207C920100F028F99B
:1044100000F09AF810BD074BE2899A42FAD10120C8
:1044200000F01EF80021207C00F0FAF8F0E7C0460A
:104430008863FF1F8305000010B5084B1A7C002A13
:1044400009D05B69002B06D09847041E01D0FEF707
:10445000D7FD200010BD0124F9E7C0468863FF1F87
:1044600070B500210600162006F066F8012115201F
:1044700006F062F807F078FA0400092007F0BCFAA9
:1044800000222B4B2B4DDA6661321A6019685B3AB9
:104490009143002E28D0023A0A431A60AC4209D157
:1044A0000A22DA6107321A6200221A639A63013221
:1044B000DA6370BD204A944203D11E22DA610532CC
:1044C000F1E71E4A944203D13022DA610632EAE76C
:1044D0001B4A944203D14322DA610832E3E7194AC6
:1044E0009442E1D16922F7E702220A431A60462288
:1044F000AC4203D0104A944204D194225A6106324D
:104500009A61D1E70D4A944201D1E622F6E70C4ABE
:10451000944204D13422FF325A610D32F0E7094A45
:104520009442C1D1E62252005A610A32E8E7C046FD
:10453000005000400024F4000048E801006CDC0258
:104540000090D00300D8B80510B50024064B092010
:10455000DC6607F0D1FA2100162005F081FF21006A
:10456000152005F07DFF10BD00500040F8B51C007F
:104570000023134D0F00EB666860160007F0ECFB9C
:1045800001238022EB6623002F615200013B08D2F9
:1045900007F09AFA08200B4A1168002C03D120007A
:1045A000F8BD2A61F2E72B6F034203D02B69013C6F
:1045B0003370013613685B1A032BEED90124EEE742
:1045C000005000406008FF1F002370B5124D14001A
:1045D000EB6668600E0007F0BFFB01238022EB66EC
:1045E00023005200013B08D207F06EFA08200B4A64
:1045F0001168002C03D1200070BD2A61F2E72B6FF7
:10460000034203D02B69013C3370013613685B1AF7
:10461000032BEED90124EEE7005000406008FF1F95
:10462000002370B50C4C0D00E366606007F094FB4E
:104630000123E366256107F047FA8020074A8000DE
:104640001168636B034205D113685B1A032BF8D919
:10465000012070BD0020FCE7005000406008FF1FF3
:10466000002370B5134C0E00E3666060150007F080
:1046700073FB0123E36626610F33626B1A42FCD0A1
:104680002B0A23611023626B1A42FCD0EDB2256124
:1046900007F01AFA8020084A80001168636B034211
:1046A00005D113685B1A032BF8D9012070BD0020D7
:1046B000FCE7C046005000406008FF1F002370B5B3
:1046C000124D0C00EB666860160007F045FB0123F5
:1046D000A619EB660F33B4420ED107F0F5F980202E
:1046E0000B4A800011686B6B03420CD113685B1A94
:1046F000032BF8D9012070BD22782A616A6B1A4217
:10470000FCD00134E7E70020F5E7C0460050004048
:104710006008FF1F10B5084CE368002B06D1074B5B
:104720001B680A336360064B1B68236007F014F9AB
:104730000002000AA06010BDC863FF1FC8F000405F
:10474000CCF0004010B50D4B986A9A6A8242FBD1BA
:104750000B4A516894684118091B4B1E844200D3D0
:104760000B0011689060D80B5B0440185B0C106064
:104770005360044A1360044B186010BD00F0004001
:10478000C863FF1FC8F00040CCF0004010B51B4BC1
:104790001A793F2A01D93F221A711979184A194802
:1047A000117018221849028018480A8002804A8035
:1047B0009A791748802402800C208A800132424373
:1047C0002401101CA24200D9201C124AC88010806B
:1047D0005A79002A01D101325A711A7A012A01D874
:1047E00002221A725A791B7A0B4853430A21584302
:1047F00006F082FF094C206010BDC046BC63FF1F5D
:10480000480AFF1FFC43FF1FC845FF1FFA43FF1F55
:10481000A865FF1FF843FF1F71020000AC63FF1F74
:10482000F8B509210020FEF7D1FD114C011E114DF4
:1048300009D10C22104BC1CBC1C4280007F05CFA8F
:10484000FFF7A4FFF8BD0C2220000C49FEF792FDF3
:104850000C2802D0084B43CB43C40C222800084943
:10486000FEF788FD0C28EBD00C220021E5E7C046BE
:10487000BC63FF1F8863FF1F64BE0011FC0C0000B7
:10488000F50C0000F0B5002504000E0085B0AA422A
:104890006AD04B1C087801934B78897837790902E4
:1048A0001943F3783F061B040B431F430397207003
:1048B0006570262800D192E01CD8102812D807F085
:1048C0000BF94D0000013300330033009800A600BF
:1048D0009F003300330033003300330033003300D4
:1048E0003300E600232800D1C0E025285FD0FF2355
:1048F00063709BE0602800D1A3E00CD8552836D027
:1049000056284ED03328F2D109229849601C06F06F
:104910004BFF0A2528E0722800D189E0DC2800D16D
:10492000E8E0712800D179E0DB2800D0FDE0042A1E
:10493000DDD91025052A05D0551F2A003800711D24
:1049400006F032FF05223100200006F02DFF2A007C
:104950003900601D06F028FF053505E00C22200017
:10496000834906F021FF0C25280005B0F0BD013A6F
:10497000804D0C2A13D8002A0AD02800019906F08D
:1049800013FFFFF703FF0C2228007B49FEF72CFCE6
:1049900029000C22601C06F007FF0D25E4E70C221D
:1049A000EBE7744D754B2A0043CB43C2E9E7013A6C
:1049B000734D0C2A11D8002A08D00199280006F05E
:1049C000F3FE0C2228006F49FEF70EFC290013228B
:1049D000601C06F0E9FE1425C6E70C22EDE7684BE3
:1049E0002900132218001D0007F086F9FEF708FBC6
:1049F000ECE705226449601C06F0D6FE0625B3E705
:104A000012226249601C06F0CFFE1325ACE7082293
:104A10005F49601C06F0C8FE0925A5E77178F729F3
:104A200000D964E75B4B188801F092FD02259BE7F3
:104A3000594B012A03D072785A706270F6E75B789E
:104A400056E7013A554D062A0ED8002A05D001999D
:104A5000280006F0A9FE01F005F829000622601CD6
:104A600006F0A2FE07257FE70622F0E7042A04D914
:104A70004B4D2F6006F070FFA860FFF763FE042225
:104A8000039003A9601C06F08FFE05256CE7454DD9
:104A9000062AE2D906222800019906F035FE0028F0
:104AA000DBD006220199280006F07EFE06223E4950
:104AB0002800FEF799FB0123374A51780B435370C6
:104AC000CBE7931E394E1A2B0CD8551E2A0001999C
:104AD000300006F069FE3649AAB23000FEF784FBCA
:104AE00000F048F9334B31001D78601C6A1E06F057
:104AF0005BFE39E7022A00D8F9E67378BFB263702B
:104B0000B378A370032A05D0033A390092B2F01C9F
:104B1000FEF76AFB10223900E01CFEF72BFCC51CD7
:104B2000002800DB20E7607080E7DA2800D0DEE6AE
:104B3000042A00D8DBE6082A15D9B37972791B025A
:104B40001343F27912041A43337A1B0613433B6072
:104B50003B68052231002000039306F025FE042265
:104B6000601D03A956E7FE236370F1E7A063FF1FF2
:104B700070BE0011BC63FF1FFC0C000064BE00117E
:104B80008863FF1FF50C00009463FF1F7463FF1F11
:104B90003C45FF1FFE43FF1FB863FF1F9944FF1FE3
:104BA000C863FF1F6509FF1FADAC0000BB65FF1F99
:104BB000AEDE0000B965FF1F70477047020010B5F8
:104BC000094B0A32094C92B2DA815A8298811882D2
:104BD000207802F023FB0422054B012120781A7073
:104BE00007F0A2F810BDC046C644FF1F0666FF1FAF
:104BF0000566FF1F013870B5042809D806F04CFF80
:104C0000030925081200214B0221187807F08CF8BF
:104C100070BD1E4B0821187806F006FF00221C4BC1
:104C20001A72F5E700241A4B184D1A6808212878E3
:104C30001C8106F059FF2100287807F025F8012093
:104C400000F048FE00F00EFFE2E7104B0821187854
:104C500006F0EAFE0F48FFF717F90F4B0F4A9B7952
:104C6000002093800E4A13808022094B52001A8143
:104C700000F030FE00F0F6FE0A4B5B78002BC7D048
:104C8000094A136007F040F8C2E7C046D863FF1F27
:104C9000AC63FF1F0744FF1FBC63FF1FC845FF1F16
:104CA000A865FF1FB863FF1F34F0004010B501294D
:104CB00009D1054B1B78002B05D02622034B044855
:104CC0005A72FFF77BFF10BDDC65FF1FAC63FF1F4F
:104CD000C40900000300F0B50A4D8E18B14202D19C
:104CE00052008018F0BD0C782F6824093C5D0F2716
:104CF0001C700C7801313C402F683C5D5C700233C5
:104D0000ECE7C046F443FF1F0D22114B10B51A709B
:104D10000C23104C10492370093A033B0F48637071
:104D200006F042FD2D2301220D490E48A371FFF725
:104D3000D1FF01220C49FFF7CDFF01220B49FFF7FC
:104D4000C9FF00220A491000FEF74EFA10BDC04606
:104D5000D865FF1FB965FF1F23BE0011BB65FF1F8C
:104D60006709FF1FC065FF1F6609FF1F6509FF1F59
:104D7000AEDE000010B51D2207480849FEF7FAFA1A
:104D8000002805DD0922064B013018705A7010BD4D
:104D9000FFF7BAFFFBE7C046BB65FF1FAEDE0000B2
:104DA000B965FF1F10B5114B1A781870002A0ED084
:104DB00000280BD10E4B1A78062A07D85423D3406B
:104DC000DB0703D50B4B187802F028FA10BD00283A
:104DD000FCD0074B1B78012B02D0033B022BF5D8EC
:104DE000044B0121187806F09FFFEFE7DC65FF1FF9
:104DF0000566FF1F0666FF1FF8B5544E544A554915
:104E00003070082005F05EFC0121022005F058FBFF
:104E1000022005F041FC0121002005F051FB00209B
:104E200005F03AFC00F0DCFEFEF7EAF806F054FC70
:104E3000032249494948FFF74DFF2D24030004226E
:104E40001C7047490130FFF745FF30230470454D82
:104E5000454C437083702E3B062220004349EB876C
:104E6000FEF788FA062813D0200006F0FDFC022881
:104E700009D00321200006F0EFFE8D23E3706E3B86
:104E8000237119336371062220003849FEF7ACF90B
:104E9000374B1B68FC335C64FFF76CFF0020FFF7A7
:104EA00081FF344F344A0121344B1278387802F0B4
:104EB00077F9334C334B00211A783878230002F00D
:104EC0006FF901222178304B01391A7000202F4AE6
:104ED000C9B205F06BFD2E4B9B78552B31D13C228E
:104EE0002C4B5A722C4A2D4BAA81EB812A826B8261
:104EF0002021307806F0F0FE0120404205F0A2FDAE
:104F00000120404205F03EFEFFF7CEF9FEF7A0FF7C
:104F100000F094FC01204042FFF792F8012006F0D7
:104F2000CBFEF72001F0F8FA0121307806F0FCFE04
:104F3000307802F0CFFA1A4806F09EFEFEF796FE91
:104F4000F8BDFA22174B5201CEE7C046D863FF1FC7
:104F5000B94B0011AD4C00113C45FF1F7463FF1F9E
:104F60009463FF1FC644FF1F6509FF1FADAC00001F
:104F70006466FF1F0666FF1F2644FF1F0744FF1FCE
:104F8000B965FF1FD865FF1FAA65FF1FBB65FF1F1F
:104F9000B863FF1FAC63FF1FC4090000CE09000007
:104FA000DA63FF1F4A1F0000F8B50A0020230D0036
:104FB0001A40194247D04F4B1B78002B40D0FFF7C7
:104FC000C1FB4D4B4D4C4E4E99686268737A8A1AFC
:104FD000DB039A4202D36160FEF748FE327A217AFF
:104FE000531EDBB2994205D1FFF702FA002000F010
:104FF000DFFD0FE09142F9D300232372FFF71CFA83
:10500000012000F0D5FD3F4F3800FEF73DFF39008D
:1050100006F02AFE637A002B0FD0013BDBB26372ED
:10502000002B0AD1384B9B78552B01D106F06CFE32
:10503000642370795843FFF7C1FD237A013323724B
:1050400020206840F8BD0BB2002B0ADA2F4B1878ED
:1050500006F0B2FC002801D006F0B6FC8020000269
:10506000EFE70224214206D0244B01201A72FFF7F9
:1050700099FE2000E5E70B071ED5FFF763FB1E4BEB
:105080001E491F4C98684A68637A821ADB039A4269
:1050900002D34860FEF7EAFDFFF7CEF9FFF7A8F963
:1050A000012000F085FD00F0E3FB2368DB0701D55C
:1050B000FFF784F80820C4E71024214206D00D4BE6
:1050C0001B78002BD5D1FEF7D7FED2E70124214271
:1050D00007D00F4800F06AF806F07EFC00F0EAFC0A
:1050E000C7E70424080020402142ABD0FEF7C4FFEC
:1050F000BFE7C046DC65FF1FC863FF1FAC63FF1F2F
:10510000BC63FF1F0744FF1FB863FF1FD863FF1F67
:10511000EC43FF1FF0B51B4B1B4F1B883A88040064
:105120001A4E1B4D85B09A420DD832889A420AD346
:10513000184B1A882B889A4205D1174A174B1288A8
:105140001B889A421BD0052001F03CFA3B8802AA3A
:1051500013803388019053802B88114D93800F4B1F
:1051600002A91B88D3800F4B2A78188802F058FFB9
:105170000D4B08212878019A1C7006F055FD05B0EA
:10518000F0BDC046A665FF1FFC43FF1FFA43FF1F8B
:10519000A865FF1FA465FF1FA265FF1FF843FF1F3F
:1051A0000666FF1FFE43FF1FA065FF1F13B50C4BD4
:1051B0001C78002C11D1002801D00A4B18600A4A33
:1051C0000A4B11780A4A10780A4A01920A4A009258
:1051D000002205F0E3FA200016BD1124FBE7C046CB
:1051E0000566FF1F9C65FF1F0466FF1FF465FF1F18
:1051F0000666FF1FE065FF1FE465FF1F10B5064B45
:1052000012201B78052B06D1044B13221988044B5E
:10521000187801F0B3FB10BD0566FF1FFE43FF1FAA
:105220000666FF1F10B500240122114B5242187070
:10523000104B1C70104B1A8002F04CF904220F4BDB
:1052400021001A700E480C3206F0B6FC1022210024
:105250000C4806F0B1FC07220B4B1C600B4B1C707A
:105260000B4B1C700B4B1A700B4B1C7010BDC046C7
:105270000666FF1F0566FF1FFE43FF1F0466FF1F34
:10528000F465FF1FE465FF1FE065FF1FB865FF1FA2
:10529000B765FF1F0044FF1FB665FF1FF8B5174C29
:1052A0000600257806A814240078052D23D1B41F04
:1052B000134FA5B21824BD421DD88D1FADB2BD42FB
:1052C00019D8FA256D00AA4215D21D000D4F0A3DCE
:1052D000ADB2BD420FD80C4C26800C4C21800C493D
:1052E00000240A800B4A1380FFF714FF0A4B0421A5
:1052F000187806F099FB2000F8BDC0460566FF1F30
:10530000790C0000750C0000FC43FF1FFA43FF1FDF
:10531000A865FF1FF843FF1F0666FF1FF0B50BB21D
:105320000D0089B0002B00DB70E1A44E307806F050
:1053300043FB041E50D00378A22B00D122E1D02BD6
:105340001AD0912B45D143780E2B42D19C4B8288A9
:105350009A423ED19B4A83681278052A39D10320AC
:1053600018567F2835D0984B1B68002B31D05B68CE
:10537000002B2ED098472CE08078072829D806F0FB
:105380008BFB0428183F3F74A8D86378002B0CD1FE
:1053900001218C4B19708D4B1A78002A5BD08C4BF5
:1053A000307801F0FDFE002855D00722854B1A7099
:1053B00051E061780029F8D1E378002B11D0854ABB
:1053C000854B1278307801F0EBFE60706378002B2B
:1053D000EBD1200006F0F8FA80200002684009B006
:1053E000F0BD784B1B78022BF3D00121307806F00A
:1053F00043FB0028EAD10121307806F095FCE5E76F
:105400006378002BD1D16F4F032807D13B78052B50
:1054100002D101333B701EE00223FBE76F4B1A8879
:105420006F4B0293002A0BD01B78002B03D0012175
:10543000307806F0F9FB3B78062B04D1013BE9E715
:10544000029B1A70F7E7042B41D10121029B3078AF
:10545000197006F069FC5C4B1B68002BB9D01B6807
:10546000002BB6D0574A107884E76378554F002B4D
:1054700027D10622211D5B4806F096F962895A4B16
:105480005A491A80A2895A4B1A80E3890B80052158
:10549000397058490A80584A1380228A574B1A801B
:1054A000574B1B78012B09D11F2001F08BF8FA22F2
:1054B000920042430421307806F0B6FB0022484BAC
:1054C00075E7312B00D070E70022454B1A7003239B
:1054D000A0E706220021434806F06EFB0023454A60
:1054E00004211380444A30781380444A138006F024
:1054F0009BFA0821307806F097FAA379083B5A42C4
:105500005341304A03331370304B1B78002B06D0C5
:10551000334B30781A78002A06D001F07FFE012242
:10552000314B52421A8096E70121197006F0FCFBBC
:10553000F5E70821307806F077FA6378002B00D081
:1055400047E72C4B2D4F0293E388029A04211380E6
:10555000294B307803932389039A138063893B8016
:1055600006F08AFA002800D033E7264B1B68002B90
:1055700000D12EE7039902983A88098800881B68B1
:10558000984726E74379132B00D022E70389012BA4
:105590000AD11D4B1B78022B06D10821307806F06A
:1055A00043FAFFF72BFE14E7052001F00BF8082162
:1055B0000200307806F038FB0BE7C0460666FF1F96
:1055C000051400000566FF1F9C65FF1F2644FF1F92
:1055D0000744FF1FD865FF1FB965FF1FDA65FF1F6E
:1055E000DC65FF1FAB65FF1FFE43FF1FB265FF1F9A
:1055F000B465FF1FA665FF1FA465FF1FA265FF1FFF
:10560000AA65FF1F9865FF1FA065FF1F8020C001CE
:10561000014200D0E2E6CB0731D5324B1B78002B9C
:105620001DD0314E05AC3378052B1AD1023B2370C7
:105630002E4B21001B7823722D4B1B7863722D4B50
:10564000187801F051FD002809D007202A4B30704E
:105650001B68002B03D01B68002B00D0984701204B
:10566000BCE60E20254B06221B7825492370254BCE
:105670001B78637002ABC01806F096F8D8E70223D7
:1056800008001840194209D0174B1B78052B03D18D
:105690001D4B188806F0D0FA02209FE60424214210
:1056A00003D0FFF737FD200098E6082308001840D4
:1056B000194200D193E6154B1C78012C03D0022C23
:1056C0000DD008208AE6124B124A134913481B8852
:1056D0001288098800880094FFF7E0FDF1E7FFF7E2
:1056E0008DFDEEE7DC65FF1F0566FF1F0044FF1F11
:1056F000B665FF1F0666FF1F9C65FF1FB865FF1F8D
:105700000144FF1FB765FF1FFE43FF1FA065FF1F7A
:10571000F843FF1FA865FF1FFA43FF1FFC43FF1F4D
:1057200010B502A804880B20002C10D14968087815
:105730004978090201430C48814209D102211980AC
:105740000A4B59881170DB7800205BB2537010BD92
:10575000074C0A20A142FAD102211980034B9988F3
:1057600011705B79F0E7C0466E2A0000A063FF1F4E
:105770006F2A0000F7B5150008AA16884A680F4F6F
:1057800014785278120222430A24BA4214D1012218
:10579000DBB2019200962A0005F006FF041E0BD131
:1057A000074B1B68002B07D068782A78000210434B
:1057B00042425041013098472000FEBD02290000BE
:1057C0001866FF1F30B5012503790400BFB02B42D6
:1057D00027D01549408805F053FA28420DD06A4673
:1057E000124B69465B8D138002235380104B5B88FC
:1057F00093806088002202F009FB0E49608805F062
:105800003FFAC0070DD56A460B4B69461B881380CB
:1058100002235380064B9B8893806088002202F00D
:10582000F5FA3FB030BDC0461066FF1F2844FF1F89
:10583000A063FF1F0866FF1F8244FF1F10B5074CBF
:105840000749200005F0D2F92000064905F0CEF9FD
:105850000721054A054805F08BF910BDFFFF000040
:105860001066FF1F0866FF1FF0BE00112844FF1FCF
:1058700010B5024803F04CF910BDC046C5570011E1
:1058800070B55F25082607498400CA788B784001E7
:105890002A40B3433440A843234302438B70CA7069
:1058A00070BDC0469944FF1F010043B204205A0056
:1058B00002409B000C3003401A43152310B5044CE2
:1058C000E0789843143B0B4018430243E27010BD4C
:1058D0009944FF1F10B5054B082419790A00A2430B
:1058E000002801D022000A431A7110BD9944FF1FFD
:1058F00010B5054B4024D9780A00A243002801D0F6
:1059000022000A43DA7010BD9944FF1F0821F8B540
:10591000324D334BAE7804000E40AE70984204DD39
:1059200067232B70473B6B70F8BD2E4B984203DA10
:10593000E0232B703A3BF6E700232B706B7083B2A9
:105940001A0029485F3292B2284F82422CD9002C8B
:1059500003DA5B421CB204232B70053420B20A2107
:1059600005F0CAFE04B2FA239B009C4232DB0823F6
:105970002A7813432B706421200005F0BDFE0A2114
:1059800000B206F059F809B22A787B5C13432B70F9
:105990000A21200005F0B0FE0A2100B206F04CF802
:1059A00009B27B5C6A780AE06970002CDBDA5B4242
:1059B0001CB204232B70F3226B78092CE8DC134310
:1059C0006B700A21200006F037F809B27B5C1E4399
:1059D000AE70A9E7632CCEDCEDE7C0469944FF1F0B
:1059E0001B4E00001DFCFFFF2A08000017BF00111E
:1059F0000823F7B5194FCD003E7904001E403E71D3
:105A0000EDB2632806DD5F3333433B7120231D4332
:105A10007D71F7BD0300093305DA20235B42334370
:105A20003B71A623F3E70E4B019300280BDA042306
:105A3000444224B23B710A21200005F0FDFF019B86
:105A400009B25B5CE3E70928F5DD0A2105F054FEA5
:105A5000019B00B21B5C1E433E71ECE79944FF1FA3
:105A600017BF001170B50F4B1B78002B18D00E4ECE
:105A70000E4D06223100280005F046FE00280FD00A
:105A8000062231000A4C280005F08EFE0120FEF7A8
:105A9000E7FC072221003E20FEF710FEFEF754FD32
:105AA00070BDC0462366FF1F9944FF1F1D66FF1F80
:105AB0001C66FF1F10B50920FFF728FFA622024B26
:105AC0001A70FFF7CFFF10BD9944FF1FF8B51C4BAC
:105AD0003C21186805F058FF3C21040006F034F81A
:105AE00020000F003C2105F04FFF182106F02CF894
:105AF00000230E00134C0A212370300005F044FFF0
:105B0000114D0A212B5C3000637006F01DF8402215
:105B10006B5C2679A370E37838001340E3700823A8
:105B20000A211E4005F030FF2B5C0A211E4338007D
:105B3000267106F009F86B5C6371FFF793FFF8BDFF
:105B4000C863FF1F9944FF1F17BF001110B5164C03
:105B50000A210223E05E05F0CFFD00B2FFF7D6FE7A
:105B60000423E05E642105F0C7FD012100B2FFF7C8
:105B70003FFF237A0024132220009A426041C0B2E2
:105B8000FFF7B6FE0320FFF77BFE2000FFF78CFE39
:105B9000064B1878053843425841C0B2FFF79AFEC9
:105BA000FFF760FF10BDC046A063FF1F0566FF1F23
:105BB000094B10B51B689B0708D5084A1378591C78
:105BC0001170DB0704D5FFF781FF10BD0028FCD062
:105BD000FFF7BCFFF9E7C046BC63FF1FB863FF1FB8
:105BE000002010B5FEF73CFC0D223E200549FEF7D3
:105BF00065FD0023984200D13E33034A1370FEF73F
:105C0000A3FC10BD0ABF00112366FF1F0200F0B500
:105C100001270A480A4E51188B1A002B00DCF0BDF0
:105C2000082415784308684038404000805B013CF8
:105C300058406D08002CF5D10132EDE7FFFF000060
:105C400028BF0011F0B500250F269D4200DBF0BDF6
:105C50004C5D070944403440A400A0580135784009
:105C6000F3E70000F0B589B06A460D000B000F277E
:105C7000110010351C780133260024093E401670AF
:105C800054700232AB42F5D12023024AFFF7DAFF0B
:105C900009B0F0BD2CBF0011F0B54E780B7889B07B
:105CA00036020C00170001901E43012A61D9954B62
:105CB0009E4200D877E001339E421CD1062A17D1BC
:105CC000CA788B7812021A430B791B0413434A7962
:105CD00012061A438C4B5A6100221A705A808B4A62
:105CE0005A608B4A9A608B4ADA60002009B0F0BD96
:105CF00088225205EEE7884B9E423CD182498B7840
:105D0000002B00D0F6E00C2A31D10F22A378934368
:105D1000E2781202134322791204134362791206C5
:105D200013434B60E279A07912020243207A000407
:105D30001043627A12060243CA60E27AA07A120223
:105D4000024376484A81834208D804236E491422CC
:105D500001980B7005F028FD1420C7E71201D21836
:105D600089235B059A42F0D801238B70BDE7022A94
:105D7000FAD00523EAE76A4A01239642E6D1FFF703
:105D80003DFA052F0CD9E378A2781B021343227940
:105D900012041A4363791B061343624A0393136088
:105DA00005F0B2FFA1E7584D2B78002B9DD1AB78C1
:105DB000002B00D1A0E02B8901339BB20093B342AA
:105DC00000D091E0132AD4D9CF7C8B7C3F021221E2
:105DD00020001F43FFF71AFF874200D08EE0002EFD
:105DE0003DD1E378A2781B0213432279E9681204BB
:105DF0001A4363791B06134303930A228B4212D181
:105E0000FF23A370E370237163716B89002B09D1A9
:105E1000E37B227C1B0212041343A27B13431B0966
:105E200001336B8100226B89002B8ED0002A67D151
:105E3000686837013818000B6B69000303909842BB
:105E400005D9686105F050FDEB780133EB706868A7
:105E50001022A11C381805F06FFD2E8145E76F89CF
:105E6000009A7B1E9BB293423AD1E278A378120249
:105E70001A43237905A81B04134362796C68120640
:105E80001A43EB6800920392211D0C22049305F043
:105E90008BFC0120260004A940421036FFF7E2FEE9
:105EA000013F012F17D1009A0B232861824200D0B5
:105EB0004CE704221C49200005F03EFD042203A902
:105EC000686805F0C1FCE968039AFF23914200D19C
:105ED0003CE7F73B3AE73100FFF7C4FE1036DFE757
:105EE0000923B742A4D831E7009BB34200D9FCE6AE
:105EF00007232BE7022329E7032327E7062325E7C8
:105F00000A2323E7FFFE0000A044FF1F0000011149
:105F1000FFFF00005048593601FF0000FFFF00114D
:105F200002FF000034F00040AC44FF1F10B5034CEA
:105F30000B000122210000F06BFA10BDED60001192
:105F40000B8870B506000D000224162B11D92B000A
:105F50000322094900F05CFA041E0AD1074B2A8883
:105F60001B88191C934200D9111C300089B200F023
:105F7000EFFA200070BDC046196100117E66FF1F58
:105F800010B54A780400013A0B000220012A07D814
:105F90000A78002A04D005222000024900F038FACD
:105FA00010BDC046476100110A7810B50B0004000F
:105FB0000220002A04D007222000024900F028FA1B
:105FC00010BDC046F36100110A7810B50B00040043
:105FD0000220002A04D009222000024900F018FA09
:105FE00010BDC0465962001110B5034C0B000B22C6
:105FF000210000F00DFA10BD8962001110B5034CAC
:106000000B000D22210000F003FA10BDFB6200110D
:1060100010B5034C0B000F22210000F0F9F910BD60
:10602000556300110A7810B50B0004000220002A05
:1060300004D011222000024900F0EAF910BDC04648
:1060400065630011002310B51322190000F0E0F978
:1060500010BD000010B5034C0B001722210000F00A
:10606000D7F910BDB7630011002310B5192219002C
:1060700000F0CEF910BD000010B5034C0B001B2240
:10608000210000F0C5F910BDF1630011F7B5848956
:106090000D0006000121002C22D000238268D35677
:1060A0001778002B1EDA0C2C1AD90C3CA4B2131949
:1060B00040880093230002F086FE431E9841013081
:1060C0007B06DB0F6B703F23013C1F40A4B228709E
:1060D000AF70AC80002C07D0B3680133AB600021F7
:1060E0000800FEBD0020EBE7AC60F8E70B7803701A
:1060F0004B8843704B881B0A83700B79C370042054
:1061000070470420022B06D10020537811781B021F
:10611000009A0B43138070470B8803700B881B0A8F
:106120004370022070470420009983420AD15378BB
:1061300010781B0203430B80D37890781B02034333
:1061400000204B807047F8B50D004B7801240021EA
:10615000461C03702B788B4201D82000F8BD6B7869
:10616000B01C4F1C012B10D1890069184B880222EA
:1061700033704B88B9001B0A7370691805F0E4FD91
:1061800004360434A4B2F9B2E4E7122359436B187D
:106190005A88043132705B8810221B0A73706918A8
:1061A00005F0D2FD12361234ECE770B5049D1400F0
:1061B0001E00052B01D8042070BD637812781B02E5
:1061C00013432B80E378A2781B02134302226B80D7
:1061D0002A71211D681D063E05F0B6FDB2B22A8166
:1061E000F02AE8D82800A11D0A3005F0ADFD0020F6
:1061F000E2E7002310B50A789A4201D8900010BD5A
:106200009A008A185488013304705488DBB2240A37
:106210004470948884709288120AC2700430EAE74D
:1062200010B51100029C062B04D004201022142B60
:1062300001D010BD022222714B7808781B02034363
:106240002380CB7888781B02034363800431601D70
:1062500005F07AFD0020ECE710B50C788B7804315E
:106260005C43E4B203702200013005F06DFD601C58
:1062700010BD0420022B06D10020537811781B0298
:10628000009A0B431380704710B50C000A88023146
:1062900005F05AFD208810BD70B504000D0004986B
:1062A0001100012B01D8042070BD1678527812021B
:1062B000324302800200F83255701470E825002C39
:1062C00000D10C35023B9AB24280AA42EBD802318F
:1062D000043005F039FD0020E6E7042000998342F0
:1062E0000AD1537810781B0203430B80D37890783F
:1062F0001B02034300204B80704710B50C000A8836
:10630000023105F021FD208810BD000070B501218B
:106310001E000420049C0E400B4218D1CB40DDB27D
:106320008D4214D90A49DBB2098899420FD3230060
:10633000F6331D703300580011184978165C0902B5
:10634000314301332152D9B28D42F4D8002070BDBF
:10635000C044FF1F10B50C000A88023105F0F4FCA0
:10636000208810BD10B50C788B7804315C43E4B202
:1063700003702200013005F0E7FC601C10BD10B571
:1063800011000298032B01D8042010BD1478527814
:10639000043B120222430280CA788C781202224304
:1063A00042809AB28280F22AEED80431063005F09B
:1063B000CBFC0020E9E710B50C000B8803700B88BC
:1063C0001B0A43704B8883704B881B0AC3708A88F2
:1063D0000430063105F0B8FCA088043080B210BD4E
:1063E0000420012B03D100201378009A137070470A
:1063F00010B50C000B8803700B881B0A43704A8889
:106400000230043105F0A0FC6088023080B210BD7B
:10641000F0B589B003931E4B029242000700D05A98
:10642000019102F020F81325061E2DD0029B0124B5
:106430000370019B002B04D00019039998470019A1
:1064400084B26B461B7A5BB2002B0FDA1021380046
:1064500002F01CFB1925002813D130003219E1B2DB
:1064600002F066FC051E0CD10C34A4B2042304AA6D
:10647000380005A993800696948101F0AFFD051EB2
:1064800002D0300005F038FA280009B0F0BDC0464F
:106490007C66FF1F70B505000C0000280CD00020A2
:1064A000814209D010222000044905F04DFC012052
:1064B0002B7823736B78637370BDC0466CBF00117B
:1064C000F0B506000D0017001C0085B002291BD096
:1064D0000020102907D1022B07D0102B03D115E083
:1064E0000020102C08D005B0F0BD69463800FFF739
:1064F000D1FF2A0069460BE069463000FFF7CAFF6A
:1065000022006946380004E0022BE9D12A00390054
:10651000300005F071F9E6E7031CF72800D9F723EE
:10652000032008499AB2013A0B80D3170340064969
:106530009B189B100B80D30F04499B185B100B809A
:106540007047C046C444FF1FC244FF1FC044FF1F22
:10655000034B1B888B4202D3024B4000C152704751
:10656000C444FF1F7C66FF1F014B4000185A704750
:106570007C66FF1F1722014B1A8070477C66FF1F45
:1065800070B505000E2005F0FFF8041E13D0D023CF
:10659000037000230622837007494570033005F01D
:1065A000D3FB064B2100DA8A62811B7E2373044BE6
:1065B000187805F031FA70BD9866FF1F8866FF1FD6
:1065C0001445FF1F262803D8024B4000C05A7047CD
:1065D0000148FCE7C644FF1FFFFF000070B506003E
:1065E0000C00094D1C220021280005F0E5FA074B9C
:1065F0001E70074B1C7005F0B7FA0123002801D06C
:10660000002312202B7070BD8866FF1F1445FF1FEA
:10661000A966FF1F70B505000D4C0800E260A1607F
:1066200010220021656005F037FB012803D11021FD
:10663000A06802F058FD10220021280005F02CFB74
:10664000012803D11021606802F04DFD70BDC046E5
:106650008866FF1F70B5041E05D1002903D00622ED
:106660000D4805F071FB0D4B1D78012D11D1002C4B
:1066700005D102221A7005F04FF8280070BD0022E3
:106680001A70074B1B78FF2BF7D02000FFF778FF1D
:10669000F3E70025F1E7C0469866FF1F8866FF1FF5
:1066A0001445FF1F030010B5002801D1002010BDC4
:1066B00000780B4A002803D15988D1821B791376C0
:1066C0001378022BF2D10023984200D103331370C8
:1066D000044B1B78FF2B01D0FFF752FF0120E6E7A8
:1066E0008866FF1F1445FF1F002911D000280CD019
:1066F0004B79012803D140225242134303E03F2249
:106700001340032802D001204B7170474022F4E768
:106710000800FAE770B5094D0100287800280BD071
:10672000074C0622200005F00FFB21002878FFF718
:10673000DBFF200004F0C8FF70BDC046A866FF1F45
:106740008266FF1F00290AD0012808D13F224B7919
:106750009343C02B03D0403B5A425341981C70478F
:1067600070B5174D06002B78FF2B15D00A2005F0C9
:106770000BF8041E10D0D0230370C83B8370114B5C
:1067800011491B784670C3700622043005F0DCFA0C
:106790002100287805F040F90C4B1B78012B0DD116
:1067A0000B4B1B68002B03D09B68002B00D0984735
:1067B000084B04211878084A05F096F970BDC046C8
:1067C0001445FF1FA866FF1F8266FF1FA466FF1FF8
:1067D000D066FF1FD466FF1F60EA0000014B986877
:1067E0007047C0468866FF1F014BDB68186870471A
:1067F0008866FF1F074B10B5DA6813680133136012
:10680000054B1878FF2803D08021C90105F08CFAC8
:1068100010BDC0468866FF1F1445FF1FF7B50E0068
:1068200002F0C8F8051E1CD00E4B06621F78002F20
:1068300000D10778AB791020019304F0A5FF041E66
:106840000FD0D0230380C73B8370019BE91DC37029
:106850000622043005F078FA21003800E66005F0E1
:10686000DBF8F7BD1245FF1F014B18787047C04693
:10687000A866FF1F054B002805D1054B1A78054B6C
:10688000002A00D1014B18007047C0469866FF1FD0
:10689000A866FF1F8266FF1F014B58687047C046FD
:1068A0008866FF1F024B1868431E9841C0B27047AC
:1068B000AC66FF1F421E03000120152A03D9FF3BCF
:1068C0005A425341D8B27047F0B51C0000230E0065
:1068D00085B0039002920B70029A934201D300207C
:1068E00019E0E55C5A1CD2B2002DF8D0029851197B
:1068F0008142F4DC0233DFB2A35C18000193FFF79E
:10690000D9FF002807D0013D019A0399EBB23370FB
:106910008A4202D1E01905B0F0BDDB19DBB2DBE73A
:1069200010B50C0002F09EF803001220002B03D0DB
:106930002100588805F020F910BD000070B50E4DFB
:1069400084006359002B15D0186A002801D005F087
:1069500023F82B59586A002801D005F01DF82B594F
:10696000986A002801D005F017F8285905F014F8A6
:1069700000232B5170BDC046B866FF1F1C4B70B57D
:1069800004000E00150099420AD11A4B1B68002B17
:1069900001D1122070BD1B68002BFAD09847F9E78F
:1069A000154B994215D1134B1B68002B0AD01B685D
:1069B000002B07D09847002804D1104B1C70104BB7
:1069C0001D70E7E729002000FFF7AAFF0028E1D1AA
:1069D000F3E7080001F0EEFF0028DAD00378032087
:1069E000A342D7D12900300005F0C6F8D2E7C0464F
:1069F000FEFF0000B466FF1FFFFF0000B166FF1F2F
:106A0000B066FF1FF7B50400808801F0D3FF0025B2
:106A1000A84203D00578A08802F008F81C4E33780D
:106A2000002B1FD0AB421DD11A4B28001978FFF75D
:106A300077FF002818D000233370A3790820A778A7
:106A4000A688019304F0A0FE011E0DD0D023037090
:106A5000CA3B8370019B477086808371280004F0D5
:106A6000DBFF01E0002DE8D1A0880B4B8200D3585A
:106A7000002B01D0FFF762FF1721A088FFF768FD08
:106A8000A08801F027FDA08801F0FEFDF7BDC046FB
:106A9000B166FF1FB066FF1FB866FF1FF0B587B075
:106AA0001D000CAB1B88070001930DAB1B88142045
:106AB00002930EAB1B88160003930FAB1B8800914B
:106AC000049310AB1B88059304F05EFE041E1AD0DD
:106AD000D0230370CB3B47708370C6700622290019
:106AE0000430002D11D005F02FF9019B21006381A6
:106AF000029B0098A381039BE381049B2382059B57
:106B0000A37404F089FF07B0F0BD05F055F8ECE779
:106B1000F7B5009308AB1B8807000C200D0016008A
:106B2000019304F031FE041E13D0280001F042FF4F
:106B300000280FD00078D0232370C93BA370009B9E
:106B400021002381019B6770A580E680638104F0AA
:106B500063FFF7BD014B1878EDE7C0461445FF1FF2
:106B600013B5040064890389C2888188C0780094C1
:106B7000FFF7CEFF13BD000010B5044C20680028BD
:106B800003D004F009FF0023236010BDBC66FF1F83
:106B9000A122F0B5818892004A43384B384F1B68D8
:106BA00004009B189D2292009B18827989B01A607C
:106BB0003B68002B5FD01D78324B1B68002B04D044
:106BC0005B68002B01D00020984726000836310072
:106BD000E079FFF7B7FD237DE0710200E0780493D0
:106BE000638A29000393238A0293E3890193A3888C
:106BF00000933300FFF752FFE378002B0BD1E289BB
:106C0000A379A18802920196E279280000920122DC
:106C100001F0DAFEE0703B68002B20D0FFF7ACFFFC
:106C2000194D287800281AD0184B1978FFF778FEEC
:106C3000002814D02B78E67808200793A78804F062
:106C4000A3FD011E09D0D0230370CA3B4670837098
:106C500087808671079804F0DFFE00232B701721D0
:106C6000A088FFF775FCA08801F034FCA08801F033
:106C70000BFD09B0F0BD064B9DE7C0463409FF1F70
:106C8000BC66FF1FD066FF1FB166FF1FB066FF1F07
:106C90001445FF1FF8B5070008000E0001F08AFE3A
:106CA000041E18D02620FFF78DFC051E00D1257884
:106CB000062004F069FD041E0DD00021062204F018
:106CC0007BFFD0232370C23B21006770A370A68096
:106CD000E8B204F0A1FEF8BDF0B585B001930AABAF
:106CE0001B78070002930BAB1B7808000D00009285
:106CF000039301F05FFE061E22D0102004F044FD35
:106D0000041E1DD01022002104F056FF2620FFF79C
:106D100059FC002800D13078D0232370C13BA370E8
:106D2000009B21002372019B67706372029BA58008
:106D3000A372039BC0B2E3720C9BE36004F06CFE91
:106D400005B0F0BDF7B50D00019001F033FE071E50
:106D500020D00E2004F018FD041E1BD02620FFF7C3
:106D600031FC061E00D13E78D0232380C53B06228D
:106D7000A370F91DE01C04F0E7FF019B2A0063816A
:106D80000123DD401A401D40210022736573F0B2DB
:106D900004F042FEF7BD0000F0B585B0029010008F
:106DA0000D0017000A9E039301F004FE041E31D06B
:106DB000029B002B2ED1039B02795B0724D5122363
:106DC00013430422002E08D10B99002905D10C99F8
:106DD000002902D10D9900291AD01A430D9B227166
:106DE000002B00D0C9E0002E00D1CFE0002D00D054
:106DF000CCE0606A002801D004F0CEFD1C213000F8
:106E000004F052FF606205E002239A430E33D7E795
:106E100093432371654BBA00D458002C00D1AAE0EB
:106E2000002E10D0236A002B03D11C2004F0ECFCB0
:106E300020625E4BBA00D358186A002803D01C2287
:106E4000310004F081FF0C9B002B12D0574CBB008B
:106E50001D596B6A002B03D1162004F0D5FC686223
:106E6000BB00E358586A002803D016220C9904F09E
:106E70006BFF0D9B002B11D04C4DBC006659B36AC3
:106E8000002B03D1142004F0BFFCB0622B59986A88
:106E9000002803D014220D9904F056FF380001F0A9
:106EA00089FD051E67D0414BBA00D358002B62D034
:106EB0001A6A3420002A00D11C389A6A002A01D0AC
:106EC000143080B20B9A002A01D01C3080B25B6A69
:106ED000002B01D0163080B204F056FC041E4AD0BC
:106EE0001822002104F068FE2620FFF76BFB0190BA
:106EF000002801D12B780193D0232370029B20001E
:106F000063700A23294EA370039BBD00A371AB5984
:106F1000A780196A1830002905D01C22A06004F04F
:106F200013FF200034307359996A002907D00300F9
:106F300014221433E060029304F006FF02980B9BC6
:106F4000002B08D003001C221C330B9920610293F4
:106F500004F0FAFE02987359596A002903D01622E8
:106F6000606104F0F1FE6B462100187904F054FDD5
:106F70003800FFF7E3FC05B0F0BD10220D9B0D9922
:106F80001B69A018236204F0DFFE2CE70B9B002B8B
:106F900000D13FE7012D00D03CE7606A002801D016
:106FA00004F0FAFC1C210B982AE7C046B866FF1FC4
:106FB00010B5044C2068002803D004F0EDFC002339
:106FC000236010BDAC66FF1F0B4B07B51A68002A83
:106FD00001D100200EBD6946531C012012780731F3
:106FE000FFF772FC0028F4D002780123100018404B
:106FF0001A42EED0EEE7C046C866FF1FF0B51F4F3D
:1070000001203B6887B0002B25D09B78059300F0CA
:10701000B3FB002821D00A20FFF7D4FA04000B208C
:10702000FFF7D0FA164B05001E78731E9E413B6891
:10703000F6B2191DD878FFF757FB3B682900DA7ABA
:10704000043303929A790193029200903300200056
:10705000059A04F0A9FD07B0F0BDFFF7B5FF0028C1
:1070600005D00620FFF7AEFA04000720D8E7082075
:10707000FFF7A8FA04000920D2E7C046AC66FF1F5C
:10708000A866FF1F70B50A4E040033780D00FF2B71
:107090000DD0042004F078FB011E08D0D02303702B
:1070A000CE3B45708370C470307804F0B5FC70BD81
:1070B0002445FF1F70B5040006200D0004F064FB9A
:1070C000011E0AD0D0230370CD3B8370054B447062
:1070D0001B688580187804F09FFC002C01D0FFF716
:1070E00067FF70BDAC66FF1FF8B5264F06003B6812
:1070F0000D001124002B05D10522234B1B781342D0
:1071000002D112242000F8BD204A10241268002A5F
:10711000F8D01278002AF5D0DB0719D52B789A1E03
:10712000012A1AD80C2004F06FFB132438600028C1
:10713000E8D000230A22437029000670023004F0D0
:1071400003FEFFF75BFF041E0AD0FFF731FFD9E70C
:1071500000F012FB0028E1D1E4E7002BE2D0D0E7F9
:107160000B4B1B78032BCDD11D20FFF72BFA094BBE
:1071700018800028C6D0084B04211878074A04F06C
:10718000B3FCBFE7AC66FF1FA966FF1FC866FF1F01
:10719000A866FF1FA666FF1FD466FF1F60EA0000F7
:1071A000F7B50193194B14001A78052306000F0058
:1071B00012201A4221D0012920D1154B1D68002D23
:1071C0001BD002201F2C18D8002C02D0019B002BB2
:1071D00013D0104B1F221E706E1C0021300004F0D3
:1071E000EBFC01992200300004F0AEFD31002000DC
:1071F0002C70002F06D004F077FDFEBD064B122048
:107200001D68DCE704F090FBF7E7C046A966FF1FA6
:10721000C866FF1F2445FF1FC466FF1FF8B50F4E49
:1072200012243368002B17D01B780F3C834213D1F4
:1072300000250B4F0221387804F0F6FB094B04219E
:1072400038781D8004F0F0FB074B28001D80336860
:107250005C7004F029FC04002000F8BDAC66FF1F40
:10726000D466FF1FC066FF1FA666FF1F70B501280A
:1072700023D11B4C2388002B03D01A4A1578002DEC
:1072800007D0194B1B68002B02D01878FFF7C6FFF8
:1072900070BD3B2B02D93C3B2380F9E7134E022102
:1072A000307804F0C1FBFA222388920002215A436D
:1072B000307804F0B9FC2580EAE70B4B1B68002B03
:1072C000E6D00B4B1B785B07E2D5084B0221187800
:1072D00004F0AAFB0022024B1A80FFF769FED7E7F1
:1072E000C066FF1FA466FF1FAC66FF1FD466FF1FAA
:1072F000A966FF1FF8B51E4D2868002803D004F0CA
:107300004BFB00232B601B4E3068002803D004F099
:1073100043FB00233360184F05243B7818002040BE
:10732000234221D0154800F02BFA3B78234213D09A
:10733000202004F069FA2860002813D020220021C0
:1073400004F03AFC202004F05FFA041E306005D0FF
:107350002022002104F030FC002004E0286804F022
:107360001BFB2C601320F8BD00F00AFAF4E7C046BE
:10737000C866FF1FC466FF1FA966FF1F1845FF1FD1
:1073800010B50A4C23681A1E0ED0002808D101300F
:10739000587004F089FB002805D02368002B02D028
:1073A0000021FFF787FE0122100010BDAC66FF1F11
:1073B000F7B5274E050033680191181E21D05C787F
:1073C000244F012C30D1FFF7FFFD002825D02000ED
:1073D000FFF7F8F80400412814D91F4B0221187850
:1073E0001E4A04F081FB1E4B3C3C1C800222336889
:1073F0005A703B78002B14D128000199FFF75AFEF0
:107400000120FEBDFA2292004243002AEED0124B28
:107410000221187804F008FCE8E7FFF7D3F802002F
:10742000F3E700233B70EBE73B78002BE8D1032028
:1074300004F0AAF9011E08D0D0230370CC3B45709C
:1074400083703368187804F0E7FAFFF7B1FDD7E7E7
:10745000AC66FF1FA466FF1FD466FF1F60EA000032
:10746000C066FF1F10B51749838802008B4220D0E9
:1074700011D815498B4217D0144900205B1899B2D6
:10748000012907D8926811785A425341D8B2FFF7C0
:10749000F9FD012010BD0E4A00209B1807229BB267
:1074A0009A424041C0B2F5E783681878FFF768FF59
:1074B000F0E7836899785A78090218781143FFF742
:1074C00077FFE7E70A20000006200000F8DFFFFF53
:1074D000AFDFFFFF014B18707047C0462545FF1F07
:1074E00010B5064C207001F041FA207804F074F9D0
:1074F0000521207800F062FD10BDC046D466FF1F54
:107500000BB273B50D00002B00DBC4E0884B18787C
:1075100004F052FA041E0ED00378912B0FD0A22B48
:1075200000D1A1E0834B1878FF2852D0210004F04D
:1075300073FA00284DD180200002684076BD437860
:107540000F2B76D013D8052B70D00E2BEAD1808864
:10755000794B98422BD8794B98421BD8784B98425C
:10756000E0D1A3681878591CFFF774F838E03E2B77
:10757000D8D18378032B74D06CD8012B6ED0022B1A
:10758000D0D1704B1B68002B23D05B68002B20D020
:1075900098471EE06C4BC0180C28C3D804F074F94F
:1075A0001DC2C2150BC20B0B0B3223C23C00674B32
:1075B000C0180728B6D8664B1B68002B09D01B687B
:1075C000002B06D0200098470AE0A3681878FFF740
:1075D000C7F8200004F0F8F9ADE7A068FFF762F8FB
:1075E00000289FD0F5E7A3681B78002BF1D0554BFE
:1075F0001B68002BEDD01B68002BEAD021005548FA
:107600009847EDE74F4B1B68002BE2D01B68002B1F
:10761000DFD021005048F3E7504B1B68002BD8D037
:107620005B68002BD5D021004348E9E7FFF7EAF972
:10763000CFE780884A4B984203D04A4B984200D00B
:1076400070E7464B1B68002BC3D05B68002BC0D093
:107650002100D5E7153B012BBBD963E7FFF798FA6B
:10766000B7E7FFF77DFAB4E73F4B1B78042B07D150
:1076700000236A4613800179408800F0C5FCA8E722
:10768000364B1B68002BA4D05B68002BA1D00100F7
:10769000364898479DE7012421420AD0294B1B68B0
:1076A000002B04D05B68002B01D0002098470120FC
:1076B00043E78B070AD5264B1B68002B04D05B6879
:1076C000002B01D020009847022036E70421280033
:1076D00008400D4200D131E7254E3388002B21D0E0
:1076E000013B9BB23380002B1AD1FFF7DBF8002857
:1076F0000AD0204B1C70164B1B68002B04D05B6813
:10770000002B01D020009847FFF7C6F8694601F02A
:1077100001FD6846FEF7FEFF1D20FEF753FF308097
:1077200004200AE7024B187804F07EF9F8E7C04617
:10773000D466FF1F2545FF1F0E200000012000001A
:1077400009100000CC66FF1FFEDFFFFFAFDFFFFF69
:10775000D066FF1F0C2000000B200000B466FF1F46
:107760000D20000013200000A966FF1FFFFF00008E
:10777000A666FF1FA466FF1F10B501F09BF910BDA0
:10778000014B18607047C046D066FF1F0B88002071
:10779000162B01D817230420014A13807047C046D6
:1077A0007E66FF1F00207047074A03001188814250
:1077B00007D091880020994202D101308000101832
:1077C00070470020FAE7C046DC66FF1FF0B58F78EF
:1077D00006000D00C7B01E2F15D1FFF7E5FF051EEF
:1077E00003D10024200047B0F0BD00223B0031004F
:1077F000C078009200F0B2FB0400A81C00F0D3FB9C
:10780000FF23EB70EEE7264B062403931B78FF2B38
:10781000E8D0182FE6D87B08224A013BDB00029211
:107820009A589446002ADDD0029AD3185B68002B40
:10783000D8D00878002802D14B78012B02D1062439
:10784000122FCFD107AFAB88697800976446AA683A
:10785000A047041EC6D1AB78029A5B08013BDB004F
:10786000D318390030005B689847041E0BD1AB7801
:10787000042BB6D0039A310010782200009700F054
:107880006DFB0400AEE76A78002AABD1AA7805A99F
:107890003B88087130000A704B80FEF747FBA0E779
:1078A0002845FF1F7CBF00111D4B37B505009842CE
:1078B0000BD000290AD1FFF777FF002805D119481E
:1078C000FFF772FF002800D0058037BD01291AD1CB
:1078D000FFF76AFF041EF8D001235B420380A37800
:1078E000FF2BF2D0FE2B07D00023E0781422009368
:1078F00029001E3300F032FBA01C00F054FB0123D2
:107900005B426380E1E70229DFD1013901F0BEF873
:107910000028DAD12800FFF747FF041EDFD1D4E7A3
:10792000FEFF0000FFFF0000022210B5074B52428D
:107930001A80074801325A809A80DA8000F07EFA75
:10794000044801F025F8002010BDC046DC66FF1F8A
:10795000CD770011A97800110388F7B50400002B3A
:1079600002D102252800FEBD426802211378254875
:107970005268FEF7A5FD00282ED0234F01253A8836
:10798000002AEFD0802321885B0201259B1A9942AF
:10799000E8DC0C2003F038FF061E31D03B8822883B
:1079A0009C4600231800019561469DB2491989B291
:1079B000AA421BD8002801D062443A80002330003C
:1079C000082208C0210004F0BFF9104A1368002BF8
:1079D00013D100251660C5E76268022113780C48B0
:1079E0005268FEF76DFD0028C7D1BAE760681D0137
:1079F0004019418101330198D6E71A001B68E6E778
:107A00001325AFE7EABF00112645FF1FD866FF1F09
:107A1000E8BF0011014B18707047C0462845FF1F92
:107A200014230A0010B51A40194204D00122102173
:107A300001F048F810BD4B06F9D4012088434000FE
:107A4000F8E710B514008B0604D50122102101F0CF
:107A500039F810BD08230A001A40194202D14BB26E
:107A6000002B0FDA102101F02DF8002808D0230098
:107A7000F9331B78002BECD0F8342378012BE8D1B4
:107A80000020E6E703208907FAD4E2E7F0B51F00FB
:107A9000184B85B01C68019002910392002C27D1ED
:107AA000200005B0F0BDA5683301ED186B89019A7F
:107AB000934211D3029A93420ED8002F04D10A9B0D
:107AC000002B10D12C00EBE73B002978039A686863
:107AD000FEF7F6FC0028F2D10136B6B2A388B34215
:107AE000E1D82468DAE7A3680A9A5B891380E9E79A
:107AF0000026F3E7D866FF1F37B50C000A884988CF
:107B00000123914217D3002A15D0651D23792A003D
:107B100002210A48FEF7D4FC102300280BD0237959
:107B20006188208800242A000094FFF7AFFF0A2311
:107B3000A04200D0230018003EBDC046EABF00119D
:107B400013B50A0008884988012388420BD8002809
:107B500009D00024137905320094FFF797FF0A2318
:107B6000A04200D02300180016BD13B50A000888F3
:107B70004988012388420BD8002809D000241379B2
:107B800005320094FFF782FF0A23A04200D02300B1
:107B9000180016BDF0B58BB003904A8808880E0017
:107BA0000123824255D3002853D00023012704AC7F
:107BB00023700022718813000092FFF767FF051EF3
:107BC0003ED02078002835D12B78022B18D1677051
:107BD0006A8983000130E31880005A8069680222B4
:107BE000201804F0B1F823780133DBB22370042BA2
:107BF00019D93B006889013080B2002BD9D01FE031
:107C000002236370122358436A89231804305A8070
:107C100069681022201804F097F823780133DBB24A
:107C20002370002BE5D10C4A6B899B185A425341B3
:107C3000DBB2DFE76378012BE4D12B78022BC7D0CE
:107C400022780A23002A04D021000398FEF798F92D
:107C5000002318000BB0F0BD0100FFFF0F4BF0B583
:107C600004001868002816D083685D89A54207D8EB
:107C70008288AE18B44203DA12019A18934201D1F5
:107C80000068EFE71E005F891036A74204D1002983
:107C900000D00D801800F0BD3300EFE7D866FF1F5D
:107CA00070B505000C0008880021FFF7D7FF03001E
:107CB0000120002B04D022002800197AFFF7C1FE12
:107CC00070BDF7B50C00002501902300F6331B783A
:107CD000AB4201D800200AE06B00E65A00213000D8
:107CE000E718FFF7BBFF002802D126800130FEBD58
:107CF000017A0198FFF794FE002802D03B88238088
:107D0000F5E70135EDB2E0E710B504000888002181
:107D1000FFF7A4FF03000120002B03D02000197AF5
:107D2000FFF77EFE10BD0000054B1B68002B01D144
:107D3000180004E09A6852898242F6D19888704708
:107D4000D866FF1FF0B50E27002687B0039302AB5D
:107D5000FF183E8005001F4B40891400984207D051
:107D60002B78013000976A6880B2FFF78FFE06001B
:107D700002212B7818486A68FEF7A2FB00280FD072
:107D80006C892000FFF7D0FF002802D0013C0419C5
:107D9000A4B2039B002B00D01C80300007B0F0BDC4
:107DA00002212B780D486A68FEF78AFB0028E7D18C
:107DB00002212B780A486A68FEF782FB002807D068
:107DC000002EDED03B88A342DBD17489013CDFE783
:107DD0006C89DEE7FFFF0000EABF0011E8BF001179
:107DE000E6BF001110B50C00FFF7DEFC0300022017
:107DF000002B0AD0002C00D023609B781720FE2B8C
:107E000003D00138FF2B00D1002010BD73B50D0049
:107E100001A904001600FFF7E5FF172805D0002E82
:107E200004D129002000FEF727F976BD0122102198
:107E3000200000F047FE0028F3D0F6E7014B186061
:107E40007047C046E866FF1F37B56B469D1D0100B1
:107E500004000222280003F0A7FC2B88B02B0ED1CF
:107E60002379122B09D12300FF339B78012B06D1F4
:107E70000121608800F0E0F801E01B2BF8D037BD4D
:107E800010B5054B0421187000F098F8FFF74CFD71
:107E9000FEF770FB10BDC046EC66FF1F0020F0B57A
:107EA0000BB20F0087B0834234DA274B187803F007
:107EB00083FD051E2BD00378A02B25D103AE310006
:107EC000FEF7E4F8041E0BD1B378DB0724D51F4B73
:107ED00006341B68002B03D03100688898470400E3
:107EE000A868002801D003F007FD002C08D1184A2B
:107EF000039B1340174A934206D0B3781B2B03D041
:107F00000121688800F098F8280003F05DFD8020CA
:107F10000002784007B0F0BD0F4B1B68002B10D05B
:107F2000310068889847041EDAD07378002BD7D1C7
:107F3000B27801A90A704B800C716888FDF7F6FFD2
:107F4000CEE70624F1E7C046EC66FF1FE466FF1F9C
:107F500000FFFF0000011200E866FF1FF7B5019067
:107F6000822040000D0017001E0003F00DFC0400ED
:107F70001320002C12D0B02320002370089BFC2279
:107F80006770658026710830002B08D0190003F057
:107F9000DBFE2100019803F03FFD0020FEBD0899A3
:107FA00003F00AFEF5E710B5041E06D00078FD28A0
:107FB00003D803F0C1FBFF23237010BD0A1F93B247
:107FC00010B504000220032B05D882400020024B8C
:107FD000D1529B189C7010BD0C67FF1F0B8870B5A9
:107FE000043B04000D000220032B0BD801212000CC
:107FF00000F04CFD03001420002B03D029002000CA
:1080000000F0DEFB70BD000007B51300034A0092CC
:108010000A00012100F02CFC0EBDC0464582001173
:1080200007B5019203220092024B0A00122100F0D0
:1080300049FC0EBDC382001107B56B4601AA118031
:108040000449D88008780633012802D1190003F0CA
:108050002BFC07BDED66FF1F0C4B10B518700023FD
:10806000FF210B4A1380138193819380094A538027
:108070001370517293819372D174D38213755177B7
:1080800003F082FD00F0FCF910BDC0461C67FF1F25
:108090000C67FF1FEE66FF1FF0B58DB06B4600202A
:1080A00003910C229B5E834200DBB0E05D4B1878AD
:1080B00003F082FC051E00D1A4E00378902B00D0D1
:1080C0009DE006AF01004688380000F013FA796899
:1080D0000400002900D19CE03B88052B6ED13B8930
:1080E000032B1CD905AC200000F0A2F86288172AE7
:1080F00061D83989131D994231D1796823780431C7
:108100000291D90738D5607800F08EF9071E06D0A5
:10811000002303712378012B08D0132B23D0A868E8
:10812000002800D178E003F0E7FB75E0628802994F
:1081300009A800F0A6F80290380000F08BF909AA0F
:108140002378387A0192002231000092029A00F0DE
:1081500012F9380000F064F9029B002BDFD03000E8
:1081600000F080F9DBE70378032BD8D1628802990D
:1081700009A800F0D6F8DEE7122B13D1029909A85E
:1081800000F0B5F8021EEAD127498B88002BC6D033
:10819000887909A92378019161780091310000F074
:1081A000EAF8BCE7002302AA93833000617809AAA9
:1081B000FFF72AFFB3E71D4B0993F6E7042B02D024
:1081C0009A1F012AABD8184A043B9B00995A0029F0
:1081D000A5D0D218907831003A0000F0AEF800280F
:1081E0009DD13B88042B03D001213000FFF724FFF1
:1081F000012C04D1A868002801D003F07DFB2800E1
:1082000003F0E2FB8020039B0002434018000DB006
:10821000F0BD012800D182E701213000FFF70CFFFB
:10822000EDE7C0461C67FF1F0C67FF1F010017002A
:108230000B7803704B784370CB788A781B0213431A
:10824000438070470A88030002700A88120A42704D
:108250000A88012A06D14A8882704A88120AC270A6
:108260000420704702208242FBD14A8804309A7071
:108270004A88120ADA708A881A718A88120A5A7130
:10828000EFE710B50400012082420CD94B780A7840
:108290001B0213432380834206D1CB788A781B02CA
:1082A00013436380002010BD022BFBD1CB788A786A
:1082B0001B02134363804B790A791B021343A3808B
:1082C000F0E70B8803700B881B0A43704B888370A0
:1082D0004B881B0AC3708B8803718B881B0A437100
:1082E000CB888371CB881B0AC371082070470300B9
:1082F0000120082A14D14A780878120202431A8011
:10830000CA788878120202435A804A7908791202A0
:1083100002439A80CA798879120202430020DA80E7
:10832000704710B504000120022A05D100204B78C7
:108330000A781B021343238010BDF8B506001020F5
:108340000F00150003F020FA04000120002C0ED0CD
:10835000A0230C22290023806780201D002D07D038
:1083600003F0F2FC2100300003F056FB0020F8BDC2
:1083700003F022FCF6E7F7B51E00009008AB1420CE
:1083800017001D78019103F0FFF9041E12D0A223FB
:108390000370019B47704380099B057146710C2255
:1083A0000830002B07D0190003F0CEFC2100009804
:1083B00003F032FBF7BD099903F0FEFBF6E737B592
:1083C000041E0FD04388002B0CD00025C188132336
:1083D000007A172201950095FFF7CDFFFF236580F6
:1083E0006372257037BD000010B50C4904004A883F
:1083F000002A09D08B89002B05D00020CB8A0222CD
:10840000834201D010BD012213000A204343002003
:108410004032C854C81842800472F3E7EE66FF1F6A
:108420000023438003707047094B00211A0010B5E8
:108430005C88002C06D01C79844203D10A234B436C
:10844000D01810BD01310A330329F1D10020F8E71B
:10845000EE66FF1F10B50400407A03F06DF9FF23AC
:10846000637210BD7047043010B580B203F064FB36
:10847000002803D00421494203F0E6FB10BD0000B0
:1084800070B50025104CA0682580A581A580A84264
:1084900002D003F031FAA56000250C4C0C4B606D46
:1084A0001D80230058331D70A84202D003F024FA27
:1084B000656500256068002801D003F01DFA0135CC
:1084C00008340A2DF6D170BDB467FF1F5867FF1F2F
:1084D000A867FF1F70B5041E09D1054D2880A8812B
:1084E000A880A868002802D003F006FAAC6070BD2E
:1084F000B467FF1FF0B54B8885B00193002343603C
:108500000A7905000F00022A00D07BE0CA88032AFE
:1085100017D98B685E7819783602DC78D8790E43E3
:1085200099781B7A24021B020C43034353495BBA1C
:108530000B80331D93421ED1042C04D0631F022BE9
:108540000ED9012015E0019A4D4B1201D35A002B90
:1085500006D00198FFF7BEFF4A4A13690133136141
:108560000421B8682E812C80494203F06DFB6860BD
:10857000002005B0F0BD434D042C06D0631F022B34
:108580000FD9EB680133EB60DBE7019A3C4B12013A
:10859000D35A002B05D00198FFF79CFF2B690133BC
:1085A0002B61374B30000293019B029A1B01019310
:1085B000002301998C468B52130063449C800393E3
:1085C0009E81FFF750FF039B041E986016D0042184
:1085D000B868494203F038FBFA880100043A2000E9
:1085E00003F0B2FB0199029AFB888A5A043B9B185C
:1085F000029A8B522B6801332B60A2E7AB690133DF
:10860000AB619EE71E4B0293019B1E01029BF35A36
:10861000002B2DD002998C19A068002828D0012A9F
:1086200026D1FA889B189BB27352A189994217D31D
:108630009B1AC018B96803F087FB029BA289F35A02
:10864000934200D07DE700222B81A3882B80A36872
:108650006B60029BF2520B4A53680133536070E720
:10866000084A9368013393600198FFF733FF68E786
:10867000044A536901335361F6E7C0461E67FF1F82
:10868000B467FF1F2467FF1F70B5051E15D10B4C83
:108690000B4B1880230058331870606D002802D0EF
:1086A00003F02AF96565250050356068002801D07F
:1086B00003F022F90834AC42F7D170BD5867FF1FB0
:1086C000A867FF1FF0B51700A12285B092000193A3
:1086D0004243394B06001B680C009B18D933FF330B
:1086E0001D78FDF741FF0430854204DD3000FDF7C1
:1086F0003BFF0430C5B2BD4207D33A000021300031
:10870000019B03F039F805B0F0BD2900380003F0F3
:108710003BF92300C6B250331E700393019B29001E
:108720006365380003F010FACBB20293002B02D03D
:10873000039B01361E7000262300503303931B78E1
:10874000B34204D8606D002831D10020DBE7029AE3
:108750002800002A04D0013B1000B34200D02800BA
:10876000F700E719387003F097F8786000280ED00A
:108770003A78019903F0E8FA019A3B780136D31868
:108780000E4A0193D369F6B20133D361D4E7039B58
:1087900018706065A74205D1084A1320D36A0133D7
:1087A000D362B0E7606803F0A7F80834F2E703F09B
:1087B000A3F800236365C8E73409FF1F2467FF1F80
:1087C000F7B50D0007000421686803F03DFA2B8916
:1087D000040003702B891B0A43702B8883702B883D
:1087E0001B0AC3702E8902250436F6B2FB2E15D85B
:1087F0001B4B9F4214D10C2002F0C6FF1135011E05
:108800000CD0902303708E3B0371043B4380154BC7
:108810008460C680187803F0FFF800252800FEBDAC
:108820005C237B43104AD3180093583301931B7881
:10883000002B0FD10300320038000099FFF742FFF0
:10884000019B05001B78002BE8D13800009903F04C
:108850000BF9E3E7054A0725536A01335362DDE765
:10886000FEFF00001C67FF1F5867FF1F2467FF1FE4
:10887000F0B587B0009017200F0016000193FFF7A6
:10888000F2FD1325041E19D00C98031E02D0019985
:10889000201D9847030AE370052302AAA070043044
:1088A000908127700098667003A993800494FFF765
:1088B00087FF051E02D0200003F01EF8280007B035
:1088C000F0BD0000F0B587B01F000CAB1B78039122
:1088D000059301210DAB06001C78049200F0D6F838
:1088E0001425002821D02000FFF77EFD0135041E4D
:1088F0001BD01149059B0A7803700132D2B2131EB6
:10890000C68001D101231A000B7022713000049B34
:1089100003990097FFF7ACFF051E09D12300210042
:108920000648074A093302F05FFF280007B0F0BD90
:10893000002363802370F8E72067FF1FBF830011C7
:1089400030750000F8B505000E00064C064F236890
:10895000002B02D03100280098470434BC42F6D1E5
:10896000F8BDC046C467FF1FD867FF1F0123064A32
:108970005B425380002313715362044A13605360B7
:108980009360D36013617047D867FF1FC467FF1FF0
:108990000200002310B506499C000859002801D1A7
:1089A000625010BD0133052BF6D11320F9E7C04604
:1089B000C467FF1F034A5388181A43425841404274
:1089C00010407047D867FF1FF0B585B002930AAB1F
:1089D0001F780CAB1B88009008000E0001920393D7
:1089E000FFF7E8FF05001120002D1BD10E48FFF70F
:1089F000E1FF04001520002C14D006220B99A7716A
:108A0000E01D03F0A1F9019B30002371029B2900B6
:108A10006371009B66802370039B6562E381FFF7AF
:108A200091FF280005B0F0BDFFFF000010B5FFF773
:108A3000C1FF04000220002C12D060880121FFF742
:108A400081FF606A002801D002F0A6FF28220021E1
:108A5000200003F0B1F8012300205B426380207105
:108A600010BD000030B5074A074C55880100137847
:108A70000020A54204D05B1A59424B415842104095
:108A800030BDC046D867FF1FFFFF0000084A10B581
:108A900001230C00904208D0FFF78CFF031E04D086
:108AA000037923405A1E9341DBB2180010BDC04623
:108AB000FEFF0000024B1879431E9841C0B2704778
:108AC000D867FF1F70B504000D001600FFF772FF96
:108AD000002804D10D4B9C4200D0143070BD416A77
:108AE00003790520002907D012221A40102A02D14A
:108AF0000520002EF2D10F20DB06EFD5897E0C2059
:108B0000A9428941494249420840E7E7FEFF000087
:108B1000030010B5002800D110BD0348034A418866
:108B20009142F9D09847F7E7D867FF1FFFFF000091
:108B3000002330B5C45CCD5C6C40D4540133102BA1
:108B4000F8D130BD0F23002210B5C45C640022436D
:108B5000CA54C25CD209013BF7D210BD0200010029
:108B600010B52032103102F0FFFD10BDF0B58BB012
:108B70000390102005931700049102F045FE009029
:108B8000102002F041FE009B13240190002B05D021
:108B900000280CD11324009802F0FEFE019B002B4C
:108BA00002D0180002F0F8FE20000BB0F0BD10203B
:108BB00002F02AFE0600102002F026FE1324050013
:108BC000002E00D1AEE0002819D01022002102F0C2
:108BD000F3FF32002900039802F0C6FD041E0ED1F7
:108BE00033787F2B51D830000099FFF7ABFF009B03
:108BF0001B787F2B53D801990098FFF7A3FF300013
:108C000002F0CAFE002D02D0280002F0C5FE002CA2
:108C1000C1D1102002F0F8FD0600102002F0F4FD92
:108C20000290002E7CD0002878D03A000F3223002A
:108C30000125121105D00F333B4015B25A42534162
:108C40001BB26A1E1201002B33D0049BD2B29818BB
:108C50000099029AFFF76CFF013D102200213000BD
:108C600002F0AAFFADB2049F2D017D19AF4242D0A0
:108C7000002C33D0300002F08FFE029B002B00D17D
:108C800089E7180002F088FE85E729003000FFF729
:108C900059FF28002549009AFFF74AFFA7E7290056
:108CA0000098FFF74FFF28002049019AFFF740FF87
:108CB000A5E70F210F4004998A18D9B28F4208D92D
:108CC000D15C06A819540133102BF6D1029A0199F0
:108CD000C0E7791A48424141C901F2E73900300042
:108CE00006AAFFF725FF3200039806A902F03CFD13
:108CF00010370400BAE7002CBCD13000029906AA54
:108D0000FFF716FF320006A9039802F02DFD082296
:108D100004003100059803F017F8ABE71324A9E726
:108D20001324AAE7002800D06EE733E7F0BF001154
:108D3000F0B58BB00F0016000225009000283FD040
:108D4000002A3DD00B1DDBB21800029302F05CFD3F
:108D50001135041E34D0FDF747FD05003A00009997
:108D6000201D02F051FFEBB20393E3702B0CDBB23A
:108D70002F0A00936370FFB22B0E2370A77001932C
:108D8000FDF72CFD1022010006A802F03DFF210096
:108D9000029A04AB06A8FFF7E9FE051E0DD1039B5E
:108DA00008223370009B04A9B370019B7770F370A5
:108DB000301D02F029FFFDF71DFD200002F0ECFD43
:108DC00028000BB0F0BDF0B58FB00D00149E0390DD
:108DD00004920593002A03D1022420000FB0F0BDB5
:108DE000002EF9D00398FFF7E5FD1424071EF4D0F8
:108DF0007278337812021A43B3781B041343F27863
:108E000012061A43036A0192934201D30133E3D15C
:108E1000002D03D03B7901249B07DED508220021D9
:108E200006A802F0C9FE059B13240433DBB2180028
:108E3000029302F0E9FC051ECFD0059A0499043094
:108E400002F0E2FE04223100280002F0DDFE3900CB
:108E5000102210310AA802F0D7FE2900029A06ABB0
:108E60000AA8FFF783FE041E0FD1082206A908A84E
:108E700002F0CAFE0822311D08A802F0BDFC01283C
:108E800007D101990398FDF7C9FC280002F084FD81
:108E9000A3E70124F9E7000070B51C4C0500236826
:108EA000181E10D0002D14D11A78002A0CD1981C4D
:108EB000083202F049FF02F0E7FD0135002808D131
:108EC00023681D70012070BD0A331800082202F0CB
:108ED0003BFF2368002BF5D0122002F055FC061E44
:108EE0000DD0C12321680370457002311022023079
:108EF00002F02AFF23683100587802F08DFD2068C7
:108F000002F04AFD00232360DCE7C0460068FF1F33
:108F1000F8B504002020FDF755FB0D4EA700BB5906
:108F20000500002B0DD000280BD0D878FF2809D1E0
:108F300008492A000C55F35907480333611802F019
:108F400053FCF8BD290002F0EFFB0028F0D1F8E750
:108F50001C68FF1F0468FF1F69A1001170B5064D52
:108F600084006359002B05D0D87802F0E5FBFF227E
:108F70006359DA7070BDC0461C68FF1F70B50600EB
:108F80008CB00C00150000213022684602F014FE5F
:108F900031001022684602F037FE1D202100032216
:108FA000684402F031FE6846FFF7D8FD2D21040029
:108FB00003222800694402F027FE20000CB070BD97
:108FC000F0B50700160097B001931CAB1D78302256
:108FD0001EAB00910AA800211C7802F0EDFD1022C2
:108FE00039000AA802F010FE1022002102A802F0A7
:108FF000E3FD0722310002A802F006FE072202ABC1
:109000009818631E9C41019902F0FEFD02AB9C730F
:109010002B005A1E934102AAD3730021102206A8E6
:1090200002F0CAFD06221D9907A802F0EDFD1A20E4
:1090300002ABC01806221F9902F0E6FD102200992B
:109040000EA802F0E1FD102202AB0EA908781C78F0
:10905000013A6040D2B2087001330131002AF5D1E3
:109060000AA8FFF77BFD102212A904000EA802F047
:109070006BFE102206AB0EA908781D78013A6840F5
:10908000D2B2087001330131002AF5D10AA8FFF7E6
:1090900065FD044310222098E4B212A902F0B4FD49
:1090A000200017B0F0BD70B50E0014008CB00100A8
:1090B000102268461D0002F0A7FD3100082204A816
:1090C00002F0A2FD2100082206A802F09DFD6846DC
:1090D000FFF744FD04001022280008A902F094FDC7
:1090E00020000CB070BDF8B506000D000024371943
:1090F000AC4200D3F8BD02F0EFFB030A3B70631CE7
:10910000DBB201379D4203D90234F054E4B2EEE7FA
:109110001C00EDE773B506000C000225002819D0ED
:10912000002917D0032101A8FFF7DDFF6B469A79CC
:109130003F231A40013313436A463000937101A95B
:109140002200FFF71BFF051E04D10322E01C01A92A
:1091500002F0FAFD280076BD03785807DA08C00F40
:10916000D20080009B0710439B0F1843C0B270478A
:1091700007230B40C908C9000B4303707047000068
:1091800070B50400FFF7EAFE134DA4006359002BED
:1091900021D0186A002801D002F0FEFB2B59986EEE
:1091A000002801D002F0F8FB2B59D86E002801D01E
:1091B00002F0F2FB2B59186F002801D002F0ECFBF3
:1091C0002B59586F002801D002F0E6FB285902F015
:1091D000E3FB00232B5170BD1C68FF1F0E4B80006A
:1091E000C35870B50C00002B0FD09D68002D0CD01B
:1091F0002B78201D0B706B784B70A97CFFF7B8FFA4
:109200002B7E23726B69E36070BD10220021200069
:1092100002F0D2FCF8E7C0461C68FF1F014B186043
:109220007047C0461868FF1F074A03008000825835
:1092300010B5002A06D0D088984203D1012901D167
:10924000FFF79EFF10BDC0461C68FF1FF0B5264EFD
:1092500095B087000B93BB590500099112200A9223
:10926000002B31D0D888FFF7A5FB04001420002C78
:109270002AD0280010A9FFF7B1FFBB591E781D6A3C
:10928000002E23D00895FDF7EFFA07000020FDF728
:10929000F1FA0790A379E61D069310AD0CA9089882
:1092A00000F0E2FA0EA9280000F0D7FA0B9B0A9909
:1092B0000493069B09980293079B039601930097DA
:1092C0000EAB0CAAFFF77CFE15B0F0BDFDF7CCFA93
:1092D00006903000FDF7CEFAE31DA779079310AB97
:1092E00006000893DAE7C0461C68FF1F30B50C4C37
:1092F00085002A59030085B00120002A0ED01800ED
:109300006946FFF76BFF2B591A78D888054B002A5E
:1093100000D1054B6A46072100F0D9FB05B030BDEE
:109320001C68FF1F5B9800116998001130B5094C4B
:109330008500295985B010226846253102F004FDC8
:109340002A591121044BD0886A4600F0C0FB05B0B1
:1093500030BDC0461C68FF1F0599001130B5094C8F
:109360008500295985B010226846353102F0ECFCA1
:109370002A591121044BD0886A4600F0A8FB05B099
:1093800030BDC0461C68FF1F43990011F7B54D4F13
:1093900086001020F4590D0002F036FAF3592062CD
:1093A000186A132200286CD0033A29009C6802F046
:1093B000CBFCF3591A780192002A58D11E6A227DFB
:1093C000317B944651400122019F114201D16746F1
:1093D0001740217D914339432175377B4F40BC466F
:1093E00060460027800701D44F0817400121022062
:1093F0008F40227D82433A432275377B5740BC46DB
:1094000060460027400701D497080F400420227DC2
:10941000BF0082433A432275627D0027944660462E
:10942000727B42400A4201D167460F400121627DB2
:109430008A433A436275777B5740BC4660460027B3
:10944000800701D457080F400220627D7F008243CD
:1094500017436775767B00227E40760701D4BA08F1
:109460000A400426617D9200B1430A4362756A781E
:10947000002A08D06278002A05D005220533DA7761
:1094800000221000FEBD04222979114205D1A17CE1
:10949000114202D10533033AF1E7019A21782C7881
:1094A000002A02D10A002100140018220429E8D859
:1094B000042CE6D805206043034A05331218525C99
:1094C000DDE7C0461C68FF1F00C0001110B50A0090
:1094D0001121024B00F0FBFA10BDC0469F9900110C
:1094E0000B0030B587B001AD2B806B460400110036
:1094F000981D082202F028FC2A000B212000024BB4
:1095000000F0E5FA07B030BDC799001110B50A00A8
:109510001121024B00F0DBFA10BDC0461B9A00116E
:1095200013B50B0011006A4613706B460400062247
:10953000581C02F009FC6A4608212000014B00F08B
:10954000C6FA13BD3B9A001110B50A001121024B57
:1095500000F0BDFA10BDC0468B9A00117FB5050022
:109560000B4BAA00D4580800002C0FD0666F237F45
:10957000E28821780396266F0296E66E0196A46E25
:109580000094FDF709FC2800FFF7FAFD7FBDC046F7
:109590001C68FF1F10B51721FFF7E0FF10BD00008A
:1095A00070B50A000D00064B0221040000F08FFA8E
:1095B000060029782000FFF7D1FF300070BDC046BB
:1095C0006B99001170B586B000236A4613708368EA
:1095D00004001D78681E0A2859D801A902F05CFA17
:1095E000060633373B3F43474B4F5300180000F00C
:1095F00042F9062312284BD000281BD16088FFF7C0
:10960000D9F90823002813D04279002A47D1264BE4
:109610001A78072312070BD5244B1A680723002A50
:1096200006D01668002E03D0290001AAB047030017
:109630006A4613706B461B786088002B2AD1FFF7AF
:1096400067FC06B070BD180000F06CF9D4E7180094
:1096500000F087F9D0E7180000F093F9CCE7180084
:1096600000F0ADF9C8E7180000F0C3F9C4E718002E
:1096700000F0F6F9C0E7180000F0F6F9BCE71800B2
:1096800000F013FAB8E7180000F013FAB4E7072364
:109690006A46137069466088FFF782FFD1E70523A9
:1096A000012AC5D1024BB8E7A966FF1F1468FF1F46
:1096B0001868FF1FF8B52C4F8600F35904000D0001
:1096C000002B40D0DA8882423DD15A78062A33D125
:1096D0001A78002A2ED0012099681A6A097D014261
:1096E00006D0157B054203D007225A700120F8BD31
:1096F0000220014204D0157B054201D00922F4E783
:109700000420014204D0127B024201D00B22ECE77C
:10971000164B1B68002BE9D05B68002BE6D02000BD
:109720009847BB5900215B78122BDFD12000FFF74F
:1097300015FFDBE70E4BECE7112A04D1002900D01E
:1097400032252900F2E7002D08D12000FFF732F979
:10975000002803D01023027913430371210028004D
:10976000FDF798FAC2E7C0461C68FF1F1468FF1F88
:109770001868FF1F70B50E4E8500AB590400002B12
:1097800013D01B78002B11D10A4B1B68002B04D07F
:109790005B68002B01D02000984773595B78122B2F
:1097A00003D100212000FFF7D9FE70BD024BECE78A
:1097B0001C68FF1F1868FF1F1468FF1F094B8000FB
:1097C000C3581020002B0CD01A6A002A09D09B68BD
:1097D000002B06D0127A1B7E101C9A4200D9181C4E
:1097E000C0B270471C68FF1F70B503000D00140065
:1097F0000220002A30D000292ED013700B78081DCB
:1098000053704B789370FFF7A7FCE07001200221A2
:109810002B7A23716B7B034063716A7B0A4013438D
:10982000042263716E7B1640334363716E7BF608CE
:10983000F600334363712B7B0340A371287B014007
:1098400000200B43A371297B0A401343A3712A7B99
:10985000D208D2001343A37170BD10B50A000100F5
:109860000120FFF7C1FF10BD10B50A000100022062
:10987000FFF7BAFF10BD70B506000C000220002EE5
:1098800030D000292ED07378201D0B70B3784B7028
:10989000F178FFF76DFC01223579257271794B1053
:1098A000080013409340104003438810104080008C
:1098B000C9080343C9000B436373B1794B10080017
:1098C0001340934010400343881002409200C9089F
:1098D0001343C9000B4321202373FCF773FE854219
:1098E00001D2122070BD2220257AFCF76BFE854242
:1098F000F7D823781820042BF4D86378012BF1D8FB
:109900000020EFE7030010B50220002909D0002B4A
:1099100007D00322481C0A7019000D3202F014FA15
:10992000002010BD03000222080010B5002B06D055
:10993000002904D00E32591C02F006FA0022100051
:1099400010BD030010B50220002909D0002B07D05C
:109950000422481C0A7019000C3202F0F5F90020AC
:1099600010BD10B5FFF7DEFF10BD03000220002977
:1099700006D0002B04D0052200200A701B784B7003
:10998000704703000220002B08D0002906D05B7826
:1099900000200B70013B082B00D9183070470300E2
:1099A00010B50220002909D0002B07D00622481C40
:1099B0000A7019000A3202F0C7F9002010BD10B574
:1099C000FFF7B0FF10BD02000B00022010B5002908
:1099D0000ED0002A0CD007211970118859701188F7
:1099E000090A997011180822D81C02F0ADF900205C
:1099F00010BD03000A00022010B5002B0CD0002976
:109A00000AD099785878090201431180901CD91C1A
:109A1000082202F099F9002010BD030010B50220C1
:109A2000002909D0002B07D00822481C0A70190011
:109A3000921802F089F9002010BD02000B000220EC
:109A400010B500290BD0002A09D00921197011780E
:109A500018185970511C062202F076F9002010BD2A
:109A600010B5FFF75FFF10BD02000B00022010B51C
:109A7000002A09D0002907D0517819701118062240
:109A8000581C02F061F9002010BD030010B502203F
:109A9000002909D0002B07D00A22481C0A7019009F
:109AA000063202F051F9002010BD10B5FFF73AFF61
:109AB00010BD02000B00022010B5002A06D00029BC
:109AC00004D018005178FFF753FB002010BDF0B50B
:109AD00085B017001E006A46062305000800918124
:109AE0009380FEF7C0FC1324011E02900CD03800B6
:109AF000B047041E05D1280001A9FEF76FFA041E25
:109B000002D0029801F0F8FE2800FFF701FA2000C9
:109B100005B0F0BDF0B504008BB001911500002137
:109B2000102202A802F048F8334EA700B8590028C6
:109B30003CD0C388A34239D10378002B36D1427878
:109B4000062A18D102000100553235310C3006AB1F
:109B5000FFF7A9FA002829D12000FFF72FFE020005
:109B600006A902A802F0F0F8200002A901F0ACFE5C
:109B700001200BB0F0BD816E002917D00B8A112A8D
:109B800028D19D420ED101981231093A01F034FEDC
:109B9000012807D1BB5920009D6EFFF70FFE290059
:109BA0000200DEE732212000FFF7D8FC2000FEF79C
:109BB00001FF061E1BD0416A002918D00B8AAB4258
:109BC00015D108220198123101F016FE01280ED19C
:109BD000716A0AE09D42E9D108220198123101F030
:109BE0000BFE0128E2D1BB59996E8A7EB9E72000AD
:109BF00001F0FAFFBCE7C0461C68FF1FF0B56B4DD3
:109C000087007E5985B0337802900393002B00D0F3
:109C100087E0B368346A01937078062817D101226F
:109C20001B7D134202D0217B114218D10222134224
:109C300002D0217B114251D10422134203D0237B55
:109C4000134200D08BE0019B5A7DEB5991E007381D
:109C50000428F8D801F020FF032E42678300B36E7A
:109C6000002B03D11C2001F0CFFDB066EB599C6E98
:109C7000002C1CD010220021200001F09DFF029832
:109C8000FFF79CFD01002000FFF72DFA01F024FEF4
:109C90002082200008211230FFF725FA0298FFF7F2
:109CA0008DFDA076EB592100D888FFF70FFC082224
:109CB000EB591CE0B36E002B05D01A00198AF0880E
:109CC0001232FFF70DFC0222019B197DEB59114264
:109CD0003DD0207B10423AD0073208E0F488FCF7F0
:109CE000DBFD01002000FFF711FC0A22EB595A703E
:109CF000029B9C002A595378073B042B11D8D0882B
:109D0000FEF758FE00284ED0C3895A08D2182849B9
:109D1000029B0298CB542B5941180433254801F07B
:109D200063FD05B0F0BDFCF79FFD030001208342F9
:109D300001D100200393EB59DE88FCF79BFD0399CA
:109D400002003000FFF7ECFB019AEB59117D042271
:109D500011420CD0217B114209D00B22C7E7F688B3
:109D6000FCF73CFD01003000FFF7EEFB6BE7019ACA
:109D7000527D01210A4204D0607B084201D00C22AE
:109D8000B5E702210A4204D0607B084201D00E22CE
:109D9000ADE704210A4204D0627B0A4201D01022BE
:109DA000A5E71222A3E7FA225200B0E71C68FF1FC2
:109DB0002068FF1F73A1001110B5064B1A78042309
:109DC000100018401A4200D00348FFF727FA00207D
:109DD00010BDC046A966FF1F2C45FF1F70B50400CB
:109DE000FFF7D4FA051E43D12000FFF77FFA234E78
:109DF000A400A0598268937CDB0708D50321036A7D
:109E00001B790B40012B02D1017F0B430377431DCC
:109E1000D97F8B1E022B0DD8022900D00121C088CA
:109E2000FCF790FF042133591A7F59700A431A77BF
:109E3000280070BD01290CD102231022437000219B
:109E40000C3001F0B9FE305910213530FFF74BF9D5
:109E5000EEE70529ECD10223D118437010220C3013
:109E600001F072FF04233259117F0B431377EAE7A5
:109E700008251828DCD1053DDAE7C0461C68FF1F1D
:109E8000F0B58BB0059143887E4F9E00F4591500C4
:109E90000493002C15D1012902D000200BB0F0BD95
:109EA000101D57781678FFF757F9EB6832000293C8
:109EB0002B7A0499019300903B002000FCF70CFFE3
:109EC000EBE7E388049A934201D00820E6E7237881
:109ED000012B00D1D4E0059B581E092800D9CFE002
:109EE00001F0DAFD05CE0A29CC506C859AB2290022
:109EF0000498FFF773FFD1E72000290010224530B6
:109F000001F022FFB9594B78042B02D1013B4B7071
:109F1000C3E70B000A00253335320C310498FFF7F4
:109F200095F90498FFF702FA0522431E9841BB59A0
:109F3000C0005A70B2E7200029001022553001F00D
:109F400003FF049B4F4C9D00295904980A0006AB5F
:109F500055320C31FFF77AF929591022453106A8FC
:109F600001F04AFC012808D10498FFF7F7F90590A1
:109F7000002804D106222B595A7005988EE7082331
:109F80000593FAE763780C2B7AD1E36E002B03D1AB
:109F90001C2001F039FCE066BB59D86E00286FD058
:109FA0001022290001F0D0FEBB590498DC6EFFF7A7
:109FB00005FC0D22A076BB595A706EE7E06E0028B2
:109FC0005ED063780D2B5BD12B8808220382A91CFD
:109FD000123001F0B9FEBB599A68517D022211423C
:109FE00026D0186A407B104222D00C32E4E7637816
:109FF0000E2B45D1236F002B03D1162001F004FC5A
:10A000002067BB59186F002803D01022290001F0E7
:10A010009BFE0F22BB59CFE763780F2B30D1206F07
:10A020000622691C103001F08FFEBB599A68517DE1
:10A030000422114203D0196A497B1142D5D1002173
:10A040000498FFF78BFA28E7636F002B0DD0BB59FC
:10A05000586F0028F3D01022290001F075FE01226C
:10A06000BB5952425B6F1A61E9E7142001F0CCFB47
:10A07000BB5960675B6F002BE9D126E72978DFE7E2
:10A0800007200BE71C68FF1F10B5064C207001F07D
:10A09000A3FD06212078FDF791FF0348FEF778FC29
:10A0A00010BDC0462F68FF1F2992001100200BB27F
:10A0B00070B50D00834216DA264B187801F07CFC4F
:10A0C000041E0DD00378922B0ED0A02B37D0224B3C
:10A0D0001878FF283AD0210001F09EFC002835D1E5
:10A0E00080200002684070BD43780E2B0BD03E2BC1
:10A0F000EDD18378052B12D0082BE8D181798088A7
:10A10000FFF7D8FA08E0154B82889A42DFD18368BE
:10A110001878591CFEF7C0FE002817D1D7E7104B5E
:10A120001B785B0712D50F4B1B68002B0ED09B686A
:10A13000002B0BD0C289811D80889847ECE7FFF780
:10A1400041FAA068002801D001F0D6FB200001F000
:10A150003BFCC5E72F68FF1F2545FF1F18200000A7
:10A16000A966FF1F1868FF1F10B50078FFF712FAE5
:10A1700010BD10B50078FFF7FDFA10BD0C23434366
:10A18000084A10B59B185A68002A03D0012901D14A
:10A19000904710BD9B68002BFBD00029F9D1984750
:10A1A000F7E7C0464C68FF1F10B5162813D80123E7
:10A1B0008340094A946B1C439463506B98435063EB
:10A1C000D46B20009843012901D120001843D063AB
:10A1D000116B0B43136310BD00800040F0B50024E9
:10A1E0000127154B85B0DA6B144E03921A6C01925D
:10A1F000DA64019BE3403B4217D0039DE5403D40BC
:10A200000295E5B202992800FFF7B8FF316A736A38
:10A21000002908D03900002B01D00299794028008C
:10A22000FFF7C2FF01E0002BF9D101340C36172CE7
:10A23000DFD105B0F0BDC046008000403068FF1F90
:10A2400010B5012402002000162A08D8054B5968D1
:10A25000D140214204D01868D0400123184010BDDD
:10A26000186DF9E700800040162807D80122064B38
:10A270008240002903D0D9680A43DA607047D96860
:10A280009143D960FAE7C0460038004030B516283F
:10A2900018D8032444430F4BE25C1B199C785D786B
:10A2A00001232D1B0135AB40013BA340A140DB4303
:10A2B0000C00122807D8084992005218116819405A
:10A2C0002143116030BD054A11680B4023431360E0
:10A2D000F8E7C04647C0001108F0004014F0004005
:10A2E000C21F70B5D4B20623092C0BD80125084C27
:10A2F0009540002908D00021FFF7C8FF23682B43B1
:10A3000023600023180070BD2368AB43F8E7C04604
:10A3100000380040F0B5162826D8214B1B185B7872
:10A32000022B21D1032444431E4A1F4EA35C121961
:10A330009478012215008540B76B013CE4B23D439F
:10A34000A240B563194C122815D89B0000290CD1E6
:10A3500017495B1899680A439A600123205C154AE3
:10A36000834011680B431360F0BD11495B18996875
:10A3700091439960F1E70E4B00290DD159690A43C9
:10A380005A61225C1328E8D00123203A93400A49FD
:10A39000086803430B60E7E7596991435961F0E7A7
:10A3A0003068FF1F47C00011008000408CC00011C2
:10A3B00000F00040A0F00040A4F00040F8B50024F8
:10A3C0001B4E1C4D1C4B1B5D012B1FD1184A926963
:10A3D000E2401A420BD00122AA5693402200143ABE
:10A3E000D2B2022A09D815494A6913434B61013494
:10A3F0000C360235172CE5D1F8BD0022AA560F49BC
:10A400009200521891680B439360F0E7022BEED153
:10A41000E7B23800FFF714FF01235840C1B23800FB
:10A42000FFF778FF3800FFF70BFF7077DFE7C046D4
:10A430003068FF1F19C000113168FF1F00F0004095
:10A44000012202388240054B002903D059690A4392
:10A450005A617047596991435961FAE700380040E1
:10A4600070B504000D000520162C1AD8002120001C
:10A47000FFF7FAFEA31E012B03D801212000FFF7EE
:10A48000DFFF00212000FFF72BFF01220A49A24035
:10A490000A4B4868012D05D102431B194A605D70C3
:10A4A000002070BD9043486002211C1961709969B9
:10A4B00091439961F4E7C046008000403068FF1F77
:10A4C00010B516280AD80122074B8240002906D071
:10A4D00019680A431A600121FFF7C2FF10BD19680D
:10A4E00091431960F7E7C0460080004070B5050051
:10A4F0000520162D17D80C2300246B430A4A21008F
:10A500009B181C70094B28005B195C70FFF7A8FFB3
:10A510000123AB40200006490A681A430A60054936
:10A520000A689A430A6070BD4C68FF1F3068FF1FBD
:10A53000348000403080004070B504000E00FF28D9
:10A5400013D003250540FFF7D1FF084AA3089B005D
:10A550009B183F22ED00AA40AE40196820009143AD
:10A56000314319600121FFF77FFE70BD18380040AC
:10A57000F8B505000520162D25D80C246C43124B88
:10A58000E4186368002B03D1A3680D30002B1AD0A8
:10A59000022201270D4B00215B195A7028002770F9
:10A5A000FFF75EFF63681E1E08D0A3683E00002B05
:10A5B00004D02800FFF744FE4640F6B228003100E0
:10A5C000FFF7F2FD0020F8BD4C68FF1F3068FF1F49
:10A5D000F7B5C420FF222B4B80001958002491436B
:10A5E0007F3A0A431A508022274F5202274E1A60A0
:10A5F000274B1D5D002D21D0A31E012B03D8012167
:10A60000E0B2FFF71DFF012D18D11F4B9B69E340FE
:10A610002B4213D0E3B218000193FFF711FE0100A3
:10A620000198FFF74DFFE3B2143B022B1DD8012127
:10A630007156184A8D405369AB4353613B7F002BE1
:10A640000DD0E5B22800FFF793FF2800FFF7F8FDD3
:10A650007B7F0100834202D02800FFF78FFD013489
:10A660000C370236172CC3D1F7BD012100237156D8
:10A67000F3568D40074A9B009B189A68AA439A603C
:10A68000DCE7C04600E100E03068FF1F19C00011A0
:10A690003168FF1F00F0004010B504000520162CA3
:10A6A0000CD801212000FFF7DBFE0123044A002023
:10A6B00011194B70A34091690B43936110BDC046C3
:10A6C0003068FF1F70B50E0015000400FFF70EFF85
:10A6D0000C236343094A20009B189D605E60FFF7CE
:10A6E00047FFF021064B074A8900051E5A5002D049
:10A6F0002000FFF7FBFE280070BDC0464C68FF1F1E
:10A700000000FF1FDDA1001170B5134D07202C784C
:10A71000002C1FD1982221005200280001F0ECFAF1
:10A720000123C420FF222B700C4B80001C635C6350
:10A730000B4B1C605C600B4B195891437F3A0A43EA
:10A740001A50802252021A600D20074A074901F070
:10A75000F3FA200070BDC0463068FF1F0080004043
:10A76000A0F0004000E100E0D1A50011BDA3001160
:10A77000030010B50620072B09D8054A137001F015
:10A7800053F8D7210020034B034A89005A5010BDCB
:10A790005445FF1F0000FF1F151BFF1F70B51D0054
:10A7A00002240C2910D8094ACA40D2070CD5FBF75D
:10A7B00015FF041E08D1059A04992800FBF72AFF0B
:10A7C000FCF798FDFFF7F8FA200070BD12100000AA
:10A7D00030B50D7802232C009C43184201D02B4346
:10A7E0001C0008252300AB43284201D02B00234343
:10A7F00020241D00A543204201D01C4325002A230C
:10A800000D70184204D011781E3B0B43137030BDFD
:10A810000028FCD10C2113788B43F7E7F8B51D0015
:10A8200006AB1B88140007AA0E000B201778002B1C
:10A8300027D10A78022A49D14A6850781178000253
:10A84000244A08438018042840D801F025F903124F
:10A850001D1B2300F06801F0B7F9021CC0B2B8421A
:10A8600000D93A1CD2B22000F1682A8001F06CFABB
:10A8700006E00222F3681B882A8023701B0A63709B
:10A880000020F8BD0622EEE701232B80F3681B7839
:10A890002370F5E7F368002B16D008222A801A8867
:10A8A00022701A88120A62705A88A2705A88120A94
:10A8B000E2709A8822719A88120A6271DA88A2710B
:10A8C000DB881B0AE371DBE72B80D9E701202B80B3
:10A8D000D7E7C04600D6FFFFF7B516000A781D007F
:10A8E00008AB1F880C000123022A18D14A6850784F
:10A8F000117800022B4A0843801803280FD801F072
:10A90000CBF802254439E06801F05EF9C0B20723B4
:10A91000B84204D37B190193152B02DD0D231800D7
:10A92000FEBDE0682A003100C01901F00DFA6B4647
:10A9300000209B88E268D0541B4B1B68834203D0E5
:10A940001B68834200D098470023E8E70B23002FC1
:10A95000E5D1022DE2D1737832781B021343E2680D
:10A960001380114B1B68002BEED01B68002BEBD023
:10A970000120E8E70B23002FD1D1062DCED12A00EC
:10A980003100E06801F0E0F9DEE70B23002FC6D1CB
:10A99000012DC3D132787533012AC0D8E3681A700B
:10A9A000D2E7C04600D6FFFF3C6AFF1F70B50C001F
:10A9B0001500072837D801F06FF8041436361B3617
:10A9C000242E182015290BD8184E162200213000ED
:10A9D00001F0F2F822002900300001F0B5F9002062
:10A9E00070BD18200229FBD11288114B1A80F6E79E
:10A9F00018200829F4D10A000E48290000F0D4FEDE
:10AA0000EDE718200129EBD10B4B10780B49DA69DF
:10AA1000FFF7DEFEE3E718200129E1D1064B1078AD
:10AA20000749DA6BF4E70220DAE7C046246AFF1F21
:10AA3000D245FF1FC845FF1F5845FF1F8045FF1F18
:10AA4000A045FF1F030010B50020DB0704D5072138
:10AA5000024A034800F08CF810BDC046A4C00011A3
:10AA60005845FF1F054A03001068002803D082885C
:10AA70009A4201D1806870470068F6E7406CFF1F7A
:10AA80000A88030008009A4204D08A8804309A4257
:10AA900000D0002070470000F8B5F82200230D4FC9
:10AAA0000D4E7968050042433370994200D07B60B7
:10AAB0000A4C0021200001F07FF800231A007C607E
:10AAC000AB4202D100203370F8BD01332280DBB2EB
:10AAD000F834F5E7406DFF1F3C6DFF1F446CFF1F0E
:10AAE00073B56B4601900600684615001980FCF7A7
:10AAF00033FF041E11D1002D0FD07689002E11D006
:10AB00000C2000F081FE00280ED0084A0460136873
:10AB100086808560002B02D11060200076BD1A006F
:10AB20001B68F7E70224F8E71324F6E7406CFF1FE1
:10AB3000012100220A4B10B549420A4C1980998024
:10AB40009A719A70084B2070012019805A60FFF7A3
:10AB5000A3FF2078FCF75EFF0448FDF719FF10BD46
:10AB6000446AFF1F486DFF1F406DFF1F1DAC0011A1
:10AB7000022310B5002802D0FFF7B2FF030018002F
:10AB800010BD0000030010B50020DB0704D5042130
:10AB9000024A0348FFF7A4FF10BDC046B8C0001129
:10ABA000D845FF1FF0B50E2687B003930CAB1F8866
:10ABB00002ABF6180500080031000292FDF74EF8CE
:10ABC00004000120002C0FD03088FFF74BFF03005A
:10ABD0000E20002B08D05E68002E05D02100280032
:10ABE000039B029A0097B04707B0F0BD0A4B10B51F
:10ABF000984207D10122002352420A808B708A803A
:10AC00008B7110BDFFF73CFF0028FAD001235B4297
:10AC1000038000238370F4E7FFFF0000F8B5050010
:10AC200001290AD1134E00243388F827AB4219D0EA
:10AC300028001149FFF7DAFF06E0022904D10139A3
:10AC4000FDF724FF0028EDD0F8BD3B006343726898
:10AC5000D018D35A002B09D03A00002100F0ACFFE5
:10AC60000134E4B2054B1B78A342EED801235B42CA
:10AC70003380DDE7406DFF1F446AFF1F3C6DFF1FFF
:10AC800010B5FFF7FDFE03000020834200D0987846
:10AC900010BD0000F0B589B01C000EAB80CB039056
:10ACA0001E8810AB1B78049202930B7A0D00DB0612
:10ACB00016D42B780593022B24D00498FFF7D2FEEC
:10ACC000002812D003689C46002B0ED0029B220065
:10ACD000019329003B00644603980096A04705E0D5
:10ACE0000498FFF7BFFE002802D10E2009B0F0BD86
:10ACF0008368002BF9D00A2229000398984700287E
:10AD0000D7D0F3E76B6858781A786B4B0002104382
:10AD10009842D2D8043B984210D2684B984242D015
:10AD200015D8674BC0180128C7D80B20002EDDD1DD
:10AD3000EB681A7859683A80200028E0614BC01807
:10AD4000032800D979E000F0A7FE846A789E5E4B64
:10AD50009842B2D10B20002EC8D101233B80EB6872
:10AD600031001B7823706889013080B2FCF776FFD0
:10AD70003A88031E0ED0017802328A183A8042893E
:10AD800062704289120AA27059680278E01C00F0D1
:10AD9000DBFF06E004323A8031000422601C00F040
:10ADA0000BFF0020A2E70B20002E9FD1EB6807A924
:10ADB0001E8804233B80330A300026706370FCF742
:10ADC0004DFF051E28D004AB9A890E2304A95B18F9
:10ADD0003E49C668FCF7B6FF00280BD12B783C48EB
:10ADE0006A680599FBF76CFB002803D1012304AACC
:10ADF0005B42D3813278022A06D17168201D00F0AF
:10AE0000A3FF3B8802333B800E2304AA9B181B88B8
:10AE1000A3701B0AE370C4E704ABDE81F4E70B20E8
:10AE2000002E00D062E7E9680398FFF729FF0223AC
:10AE30003B802070000A6070B3E70B20002E00D02A
:10AE400054E70222EB681B883A8023701B0A637068
:10AE5000A7E7E86800F0B8FEC2B203000720B242DC
:10AE600000D243E70DD00299DBB27118994202DBA0
:10AE7000921BD3B20293029BE9681A003B808919A6
:10AE80005AE70023F6E70B20002E00D02EE707221A
:10AE9000EB683A801A7822705A7862705A88A270E9
:10AEA0005A88120AE2701A792271DA886271DB8894
:10AEB0001B0AA37175E7C0460429000002280000A0
:10AEC00000D8FFFFFFD6FFFF03280000FFFF0000B0
:10AED000E8BF0011F0B58DB06B460020089120222C
:10AEE0009B5E83423DDAA64B187800F065FD071E95
:10AEF00032D00378B02B2CD10079023816281FD815
:10AF000000F0EAFD17001E001E001E0031001E00AA
:10AF100096001E001D011E0052011E0073011E003E
:10AF2000CD011E0050021E001E001E008E021E00DB
:10AF3000E302944B94491B8878880B80FBF700F858
:10AF40003800FCF781FF914B1B68002B01D03800C3
:10AF50009847380000F038FD8020089B00024340ED
:10AF600018000DB0F0BDF6220021874800F024FE45
:10AF70000BAA3B7B7989388900923A000D32FCF7A5
:10AF800085FD0400804B1B78002C3FD146E0804BB0
:10AF9000788805937F4B4100CB5A0BAE073BDBB261
:10AFA00032880293002301937B4B21000693009388
:10AFB000059BFFF76FFE744D002810D1069B3A8A5F
:10AFC0001B889A420BD138000599123000F014FC0E
:10AFD000002804D02B7862899B00EB185A80162336
:10AFE00006A81B18328820007989FCF7ABFE2B7865
:10AFF00004009A00AA1851880029C3D00133DBB29B
:10B000002B70002807D006A9C98A9180634A12884C
:10B010009A42BCD802E0012149429180002B04D021
:10B0200059497888FAF7C0FF8AE73E890A2479E00F
:10B0300000253E89574B06937B88069A5B009B5AF6
:10B04000033B9D4202DB002DF0D05BE0162206A8F8
:10B0500012183B7B798900923A0030000D32FCF7E0
:10B0600015FD0590002858D04689017A7888FCF7AC
:10B07000D7FC041E44D1464B78880793069B4100B9
:10B08000C95A454B0439C9B206AAD28A069302911D
:10B09000019400930599079BFFF7FCFD041E2FD137
:10B0A000069B39491A88931C002D26D14B8079883C
:10B0B000384B4900CB5A5119033B8B4220DD059B8D
:10B0C00031485B8941190B71A91C0135C9B2EDB238
:10B0D000059145191B0A2B71059B2D49043318183E
:10B0E00000F032FE2C4B059A1B88D318DDB22C4B96
:10B0F0009E4205D00136B6B29CE749889942D6D027
:10B10000002D0CD0204C2800618800F0F5FA20704A
:10B1100021007888FAF758FF12E7059CF0E7002C29
:10B1200000D183E77B78142B00D109E716493B79DE
:10B130004E800B700C717888FAF7F8FE00E7162441
:10B1400006ABE41821003889FCF788FD011E00D108
:10B15000B7E1788822880F4C45002C5B0A4D013CF2
:10B16000E4B2029400240F4B01940095FFF792FD86
:10B17000041E00D014E129007888FAF735FFDFE6D5
:10B18000486DFF1FC444FF1F4C6AFF1F406AFF1F2A
:10B19000466BFF1F7C66FF1F3C6CFF1FC244FF1FF6
:10B1A000FFFF00004E6AFF1F162406ABE4182100C3
:10B1B0003889FCF753FD011E00D182E1788822888E
:10B1C000AE4C45002C5BAE4D013CE4B202947C8950
:10B1D000AC4B01940095FFF75DFD041E00D0DFE04D
:10B1E00029007888FAF70AFFAAE60025A44B1D80FB
:10B1F0003B00FE331B78A24A78880792AB4208D9FD
:10B200009E4B12880693069943005B5A013B9A4273
:10B2100003DB0799FAF7FCFE92E616246B00FB1895
:10B22000059306ABE418059B21001889FCF716FD71
:10B23000011E03D1059B01241E8973E77888924B78
:10B240002288069C099343001B5B904E013BDBB2B6
:10B250000293002300960193099BFFF71BFD041E38
:10B2600002D0059B1E895DE77B88069A5B009B5A8E
:10B27000079A108832881218934202DC1B1A013B8D
:10B2800033807F4C023032880999001900F05CFD50
:10B290002388328801359B182380EDB2A8E70BAADA
:10B2A0003B7B7989388900923A000D32FCF7EEFB3E
:10B2B00000250590059B002B04D10A24002D00D108
:10B2C0006EE060E0059B7888197AFCF7A9FB010025
:10B2D000041E63D1694C6C4B788806940993069BD5
:10B2E0004400E45A694B063CE4B20BAE3288079343
:10B2F0000294019100930599099BFFF7CBFC041E72
:10B300004CD1079B5E491B881A1D002D30D14A8005
:10B31000059B5B4C5A8963191A716B1C9BB2E3182D
:10B32000120A1A71162306A832881B187989059803
:10B33000FCF708FDFF21AA1C2E1D03350B0005900C
:10B3400092B2B6B2ADB2002803D006ABDB8AD9B256
:10B350001B0AA218651911712B714C4D301D2A88DA
:10B360004949201800F0F0FC2B88F618B5B2A1E787
:10B370004988914207D17A8806995200525AEB18AF
:10B38000053A9A42C4DC3E4C2800618800F0FCFA81
:10B39000207021007888FAF745FED1E5002DF2D122
:10B3A0003E89BFE6162606ABF61831003889FCF751
:10B3B00055FC3D000400FF3500282DD0037A9B0684
:10B3C0000CD400227B893989788800923A000C32AB
:10B3D000FFF7E8FB041E10D03E8915E03088FFF728
:10B3E00041FB00281AD08368002B17D021001222BD
:10B3F00078889847041EE4D0EEE7AB78002B02D1A2
:10B400007888FAF71FFE0026AB78002B00D097E56E
:10B41000002C00D194E585E60124DDE70E24DBE76E
:10B42000162506ABED1829003889FCF717FC041E19
:10B4300047D0037A9B0611D4154A7B88118899421C
:10B4400003D01448814207D11380134BF8261D788E
:10B450000023D9B2A94221D30924A1E72888FFF704
:10B4600001FB00282FD08368002B2CD02100122252
:10B4700078889847041EDFD092E7C0467C66FF1F9D
:10B480004C6AFF1F4E6AFF1F466BFF1F3C6CFF1F7D
:10B49000406DFF1FFFFF00003C6DFF1F310059434F
:10B4A000546801336018615A0029D2D13C00083435
:10B4B0002100F82200F048FC21007888FAF7CAFD44
:10B4C0003EE501246CE70E246AE71D4B1A887B8851
:10B4D0009A4231D07888FAF7C7FD31E5F82305980C
:10B4E00051684343CD18C95A00291FD03B7A012B1C
:10B4F0000BD16C88AB887888AA1D0094FFF752FBAB
:10B50000041E02D000233B722E88F822002128005E
:10B5100000F052FB00232B80059B0133DBB2059327
:10B52000084B05991B78064A8B42D7D801235B420A
:10B530001380002CCED0F5E5002634000596EFE709
:10B54000406DFF1F3C6DFF1F70B504000E0015001D
:10B55000FFF796FA031E08D131000548FFF790FA6D
:10B5600003001120002B02D01C8000209D7070BDB4
:10B57000FFFF0000F8B50B4F06003B780D001400EC
:10B58000FF2B0ED00A2000F0FFF8011E09D0B123D6
:10B590000380002346800371C5800481387800F061
:10B5A0003BFAF8BD1946FF1FF7B50F0008A90600C2
:10B5B000088809A90B240988002821D10234022B0C
:10B5C0001ED1557813782D021D432B008B43019318
:10B5D0007334002B14D1FB68300019000093FFF77F
:10B5E0004FFB019C85420BD02A0030000099FFF7E9
:10B5F000ABFF041E04D12A0030007989FFF7BAFF9F
:10B600002000FEBDF0B50E7885B003900AA805882D
:10B610000120022E0DD14C682778647824023C4327
:10B62000054FBC4205D10398DBB201960095FFF7A8
:10B63000BBFF05B0F0BDC0460229000010B50400F4
:10B640000C4800F051F80C48A16B00F04DF80B4885
:10B65000E16B00F049F80A48216C00F045F8094B0D
:10B660000948196800F040F8084B1B68002B00D00F
:10B670009847FEE79EBE0011B4BE0011C3BE001184
:10B68000D2BE001104ED00E0E1BE00114C6DFF1FC1
:10B69000002307B501A80193FFF7D0FF044A05482E
:10B6A000002110B5121A00F087FAF8F783F9FEE7C7
:10B6B000506DFF1F1C46FF1F01B40248844601BCA9
:10B6C000604700BF8552010001B40248844601BCB6
:10B6D000604700BFC521000001B40248844601BC98
:10B6E000604700BF3136FF1F01B40248844601BCE9
:10B6F000604700BFE53A010001B40248844601BC3E
:10B70000604700BF350E000001B40248844601BC0A
:10B71000604700BFF30E000001B40248844601BC3C
:10B72000604700BF291C000001B40248844601BCE8
:10B73000604700BF5147010001B40248844601BC84
:10B74000604700BF1147010001B40248844601BCB4
:10B75000604700BF6932FF1F01B40248844601BC44
:10B76000604700BFC9A9000001B40248844601BC7B
:10B77000604700BFE548000001B40248844601BCB0
:10B78000604700BF5118FF1F01B40248844601BC46
:10B79000604700BF1D4D010001B40248844601BC52
:10B7A000604700BF8132FF1F01B40248844601BCDC
:10B7B000604700BF810E000001B40248844601BC0E
:10B7C000604700BF9130FF1F01B40248844601BCAE
:10B7D000604700BFA54F010001B40248844601BC88
:10B7E000604700BF5D17000001B40248844601BCF9
:10B7F000604700BFA946010001B40248844601BC6D
:10B80000604700BFCD4C010001B40248844601BC32
:10B81000604700BF3D4B010001B40248844601BCB3
:10B82000604700BFDD30FF1F01B40248844601BC01
:10B83000604700BF151BFF1F01B40248844601BCCE
:10B84000604700BFB14E000001B40248844601BC0D
:10B85000604700BFB537FF1F01B40248844601BCF2
:10B86000604700BF3D18000001B40248844601BC97
:10B87000604700BF093AFF1F01B40248844601BC7B
:10B88000604700BF4135FF1F01B40248844601BC38
:10B89000604700BFD13CFF1F01B40248844601BC91
:10B8A000604700BF017F000001B40248844601BC2C
:10B8B000604700BFE117000001B40248844601BCA4
:10B8C000604700BFE134FF1F01B40248844601BC59
:10B8D000604700BF311B000001B40248844601BC30
:10B8E000604700BF2951010001B40248844601BCF1
:10B8F000604700BF3939FF1F01B40248844601BCCC
:10B90000604700BFD949010001B40248844601BC28
:10B91000604700BFD53BFF1F01B40248844601BC0D
:10B92000604700BFADAE000001B40248844601BCD0
:10B93000604700BF5522000001B40248844601BCA4
:10B94000604700BF8538FF1F01B40248844601BC30
:10B95000604700BFED4A010001B40248844601BCC3
:10B96000604700BF156B010001B40248844601BC6A
:10B97000604700BFD1A5000001B40248844601BC65
:10B98000604700BFEDA5000001B40248844601BC39
:10B99000604700BF090E000001B40248844601BCA4
:10B9A000604700BF014C010001B40248844601BC5D
:10B9B000604700BFC95C010001B40248844601BC75
:10B9C000604700BFF54E010001B40248844601BC47
:10B9D000604700BF434D010001B40248844601BCEA
:10B9E000604700BFC51D000001B40248844601BC89
:10B9F000604700BFC132FF1F01B40248844601BC4A
:10BA0000604700BF413AFF1F01B40248844601BCB1
:10BA1000604700BFB54C010001B40248844601BC38
:10BA2000604700BF594F010001B40248844601BC81
:10BA3000604700BFB352010001B40248844601BC14
:10BA4000604700BF350E000001B40248844601BCC7
:10BA5000604700BFF539FF1F01B40248844601BCAE
:10BA6000604700BFC53F000001B40248844601BCE6
:10BA7000604700BF7D18FF1F01B40248844601BC27
:10BA8000604700BFC94A010001B40248844601BCB6
:10BA9000604700BFD91B000001B40248844601BCC6
:10BAA000604700BFE53CFF1F01B40248844601BC6B
:10BAB000604700BF691F000001B40248844601BC12
:10BAC000604700BFC13AFF1F01B40248844601BC71
:10BAD000604700BF9DA9000001B40248844601BC34
:10BAE000604700BFF93CFF1F01B40248844601BC17
:10BAF000604700BF5952010001B40248844601BCAE
:10BB0000604700BF813AFF1F01B40248844601BC70
:10BB1000604700BF4550000001B40248844601BCA4
:10BB2000604700BFA134FF1F01B40248844601BC36
:10BB3000604700BF9137FF1F01B40248844601BC33
:10BB4000604700BFE928000001B40248844601BCF8
:10BB5000604700BF090E000001B40248844601BCE2
:10BB6000604700BF2146010001B40248844601BC81
:10BB7000604700BF5125000001B40248844601BC63
:10BB8000604700BF8D12000001B40248844601BC2A
:10BB9000604700BF7918000001B40248844601BC28
:10BBA000604700BF456B010001B40248844601BCF8
:10BBB000604700BF851F000001B40248844601BCF5
:10BBC000604700BF154D010001B40248844601BC26
:10BBD000604700BFDD52010001B40248844601BC49
:10BBE000604700BFC926000001B40248844601BC7A
:10BBF000604700BF091B000001B40248844601BC35
:10BC0000604700BF2D3BFF1F01B40248844601BCC2
:10BC1000604700BF4551010001B40248844601BCA1
:10BC2000604700BF6571010001B40248844601BC51
:10BC3000604700BF8B52010001B40248844601BC3A
:10BC4000604700BF2526000001B40248844601BCBD
:10BC5000604700BF5549010001B40248844601BC59
:10BC6000604700BF055E000001B40248844601BC85
:10BC7000604700BF056A000001B40248844601BC69
:10BC8000604700BF3555000001B40248844601BC3E
:10BC9000604700BF2124000001B40248844601BC73
:10BCA000604700BF1D4B010001B40248844601BC3F
:10BCB000604700BFF94C010001B40248844601BC52
:10BCC000604700BF6DBC000001B40248844601BC5F
:10BCD000604700BF0189000001B40248844601BCEE
:10BCE000604700BF0124000001B40248844601BC43
:10BCF000604700BF4D1F000001B40248844601BCEC
:10BD0000604700BFB70E000001B40248844601BC82
:10BD1000604700BFA93BFF1F01B40248844601BC35
:10BD2000604700BFC56D010001B40248844601BCF4
:10BD3000604700BF0D52010001B40248844601BCB7
:10BD4000604700BF0933FF1F01B40248844601BCAD
:10BD5000604700BFE94C010001B40248844601BCC1
:08BD6000604700BF75A9000057
:10BD6800000201030202030304030502060207029C
:10BD7800080209030A030B030C020D020E030F034A
:10BD8800100311031303140315001600893D001155
:10BD9800BD3D00110000000002000000AABD001116
:10BDA800192A0F180A000000F1590000FD240000AC
:10BDB8004146010099800011ADA0001101750011E4
:10BDC8009D7E00111D530011D5AE0011A94F001121
:10BDD800D13F0011014100110000000016160000BB
:10BDE80002000000F4BD0011F4FFF3FFD2FC0000D4
:10BDF800CD41001100000000000000005475796179
:10BE08000056302E3900303030310067697468755B
:10BE1800622E636F6D2F7076767800544830350047
:10BE2800020000003CBE0011292A282A272A262AB7
:10BE3800252A242A0A180000E204000071020000E2
:10BE480078EC0000744000001027000060F000004B
:10BE580006640000204E0000000000000100000001
:10BE68001F501D00023CB40000011500090000002D
:10BE7800A102000030313233343536373839414287
:10BE880043444546005048592B36325858504C5573
:10BE98005330353034005B48617264206661756CDC
:10BEA800742068616E646C65725D0A004C522020D3
:10BEB800203D203078253038780A00504320202053
:10BEC8003D203078253038780A0050535220203DE4
:10BED800203078253038780A0049435352203D20D5
:10BEE8003078253038780A0021570011755700112D
:10BEF800000000000200000008BF00116F2A6E2A2F
:10BF08001A18D880F060FFFFFFFFFFFFFFFFFFF365
:10BF180003B59747D6F613F7D777E6F0A7F474007A
:10BF2800000001A0000000006410B71DC8206E3B8F
:10BF3800AC30D9269041DC76F4516B6B5861B24D28
:10BF48003C7105502083B8ED44930FF0E8A3D6D692
:10BF58008CB361CBB0C2649BD4D2D38678E20AA0FA
:10BF68001CF2BDBDFB349B5F800000800010000008
:10BF780000000000036100118D7700112761001196
:10BF8800957B0011AB6100116B7B001121620011E0
:10BF9800417B001173620011097D0011DB62001101
:10BFA800097D00110D630011C37C0011216200118D
:10BFB800F97A001199620011A17C001100000000BB
:10BFC800000000007F630011A17C0011E1630011F3
:10BFD800A5770011052A042A012A002A0229032824
:10BFE80001280028011800180000000000000000C7
:10BFF80000000000000000870101020102010102A7
:10C008000102030304010301010101010303020109
:10C0180003000D000E0010001100130014010701A9
:10C0280008010A010B011C011D0204020502070296
:10C03800080219021A021C021D0301030203170059
:10C048000201000504000807000B0A001716001D6E
:10C058001C010201010504010E0D01111001141348
:10C06800011716011A19020201020B0A020E0D022B
:10C078001110021413021716030504030807030B13
:10C088000A030E0D0001020307090A0B0E0F101117
:10C0980012141718191A1B1F202122001DA800119D
:10C0A800D9A800110000000002000000EEBF001136
:10C0B8000000000005B600110000000002000000AA
:04C0C800ECBF0011B8
:020000041FFFDC
:1000000000000000E53E0011B0BD0011ACBD0011C4
:100010002863FF1F00000000000000000000000037
:1000200000000000000000000000000000000000D0
:1000300000000000000000000000000000000000C0
:1000400000000000000000000000000000000000B0
:1000500000000000000000000000000000000000A0
:100060000000000000000000000000000000000090
:100070000000000000000000000000000000000080
:100080000000000000000000000000000000000070
:100090000000000000000000000000000000000060
:1000A0000000000000000000000000000000000050
:1000B0000000000000000000000000000000000040
:1000C0000000000000000000000000000000000030
:1000D0000000000000000000000000000000000020
:1000E0000000000000000000000000000000000010
:1000F0000000000000000000000000000000000000
:1001000000000000000000000000000000000000EF
:1001100000000000000000000000000000000000DF
:1001200000000000000000000000000000000000CF
:1001300000000000000000000000000000000000BF
:1001400000000000000000000000000000000000AF
:10015000000000000000000000000000000000009F
:10016000000000000000000000000000000000008F
:10017000000000000000000000000000000000007F
:10018000000000000000000000000000000000006F
:100190000535FF1F5533FF1FC16601000000000039
:1001A000000000000000000000000000000000004F
:1001B000000000000000000000000000000000003F
:1001C000000000000000000000000000000000002F
:1001D000000000000000000000000000000000001F
:1001E000000000000000000000000000000000000F
:1001F00000000000000000000000000000000000FF
:1002000000000000000000000000000000000000EE
:1002100000000000000000000000000000000000DE
:1002200000000000000000000000000000000000CE
:1002300000000000000000000000000000000000BE
:1002400000000000000000000000000000000000AE
:10025000000000000000000000000000000000009E
:10026000000000000000000000000000000000008E
:10027000000000000000000000000000000000007E
:10028000000000000000000000000000000000006E
:10029000000000000000000000000000000000005E
:1002A000000000000000000000000000000000004E
:1002B000000000000000000000000000000000003E
:1002C000000000000000000000000000000000002E
:1002D000000000000000000000000000000000001E
:1002E000000000000000000000000000000000000E
:1002F00000000000000000000000000000000000FE
:1003000000000000000000000000000000000000ED
:1003100000000000000000000000000000000000DD
:1003200000000000000000000000000000000000CD
:1003300000000000000000000000000000000000BD
:1003400000000000000000000000000000000000AD
:10035000000000000000000000000000000000009D
:10036000000000000000000000000000000000008D
:1003700091B6001100000000000000000000000025
:10038000000000000000000000000000000000006D
:10039000000000000000000000000000000000005D
:1003A000000000000000000000000000951AFF1F80
:1003B000000000000000000000000000000000003D
:1003C000000000000000000000000000000000002D
:1003D000000000000000000000000000000000001D
:1003E000000000000000000000000000000000000D
:1003F00000000000000000000000000000000000FD
:081838005071FF1F4118FF1F52
:10184000024981F3088802F013FB00005071FF1F6A
:1018500010B502F05DFB072804D0122808D002283A
:1018600008D010BD044A0420136B01331363F8E75A
:101870000220F6E71420F4E72467FF1FF8B50700FD
:101880000C0026002500503630785135002804D150
:101890000300287058342370F8BD2978CA00481E08
:1018A0008141A3183800A25C5B68C9B2FFF7D0FF82
:1018B00000280DD12B78DA00A218013350602B706C
:1018C0003378044A013B3370136A01331362D8E75B
:1018D0000123DFE72467FF1F5C234343074910B55B
:1018E000C9180B0058331B78012B05D1FFF7C6FF31
:1018F000034A936A0133936210BDC0465867FF1FC5
:101900002467FF1F10B502F013FA064A01211300E5
:1019100010CB4942D967044B136002F071FC2000E0
:1019200010BDC04600E100E01000100010B504003A
:1019300002F0FEF9024B1C6002F062FC10BDC046D2
:1019400000E100E010B5040002F0F2F94021094A7C
:10195000200013688B43136002F052FA01F0B4FDCB
:101960000022054B01201A60044B04321A6002F079
:101970004FFCFEE71CF00040C4F00040C0F0004007
:10198000431E5A425341A022F0B5D2015B4213409C
:10199000154D164A40019B182A18127E8BB00191F2
:1019A000002A1BD01A000832D46F0022E6B206AF1C
:1019B000E4B294420EDC2818C369002B08D00199C8
:1019C00002AA117106AA049202AA167303A89847E4
:1019D0000BB0F0BD1978B9540132EAE71A7D1A78D4
:1019E00006AB01261A70E6E7E469FF1F00400040DD
:1019F000F0B5254B04004001C25C85B0002A2BD015
:101A00001A18117E002927D0917E002924D011793F
:101A1000022921D11689D788D168F51BADB22A1CBD
:101A2000102D00D9102292B2BE4217D118180123EE
:101A300003710023C269C38003819A4206D06846BD
:101A4000032103730171029301A890470820002C21
:101A500000D0192001F034FC05B0F0BD013C654216
:101A60006C41A0256442ED012C40084D1B186419FF
:101A7000074D0633013A92B2AA42EDD01888461CAF
:101A80001E80085C2070F5E7E469FF1F00400040FD
:101A9000FFFF00000F220E4B10B59868104002386F
:101AA0000A280BD802F01EF90D0A0B0A0A110A0ABD
:101AB0000A0A060002210020FFF762FF10BD012183
:101AC000F9E70020FFF794FFF8E7DB6FF6E7C04681
:101AD000004000400F220E4B10B5986810400238AD
:101AE0000A280BD802F0FEF80E0A0B0A0A120A0A9C
:101AF0000A0A060002210120FFF742FF10BD012162
:101B00000800F9E70120FFF773FFF7E7DB6FF5E760
:101B10000090004013B5334C2378072B3DD8324B4F
:101B20001A78324B002A39D18022196852020A43AE
:101B30001A60252001F084FF20232D4A11680B43F1
:101B4000802113606B460422C905086807331042E0
:101B500028D080210422C905C86810422ED08021D7
:101B60002020C905CA688243CA6014221A701A78F4
:101B7000002A2FD18021C905C86820320243CA60DB
:101B800014221A701A78002A28D11A4B1A7D22784A
:101B90005A601D221A705932DA6013BD1A6816494C
:101BA0000A40C5E7086802430A6014221A701A78CE
:101BB000002ACED01A78013AD2B2F7E7C8680243B9
:101BC000CA6014221A7019784A1ED2B21A700029FB
:101BD000F9D1C4E71A78013AD2B2C7E71A78013AC4
:101BE000D2B2CEE75445FF1F1C46FF1F3CF0004019
:101BF0004C45FF1F00200040FFFFFEFF564B70B515
:101C00001B68012B03D1554A936D0133936502F094
:101C10000FFA534B534A1860534B544C1A6001232C
:101C2000534A1360534A13602378002B06D00622D0
:101C30005149524802F00CF900232370504A514B8D
:101C400010681B78C1B2002B0ED14F4CC0B2237864
:101C50005BB2002B4FDB237824785BB264B21B04A9
:101C600024021B191B1813600B1C50294ED950233A
:101C7000464A47491078DBB2FF2202284BD1086858
:101C8000444C454D267890432A78964254D9227880
:101C900024782E78023B5D10A31B6B435201D31AAC
:101CA00010335B111843086002F0A2FA031F012BE6
:101CB00045D83A4B1B78002B06D0394B1B78002BAC
:101CC00002D0002002F03CFAA122364B9200997813
:101CD000354B4A431B689B18832292009B181B7844
:101CE000033B012B03D8AF20400002F051F8012242
:101CF0002E4BDA8270BD237824785BB264B2FF3356
:101D0000FF341B0424021B190138ABE7CAB2022AB4
:101D1000AED20223ACE70868254C264D26789043C6
:101D20002A78964208D9227824782D78023B5B10D5
:101D3000641B63435201B2E72378DBB2B2E70228A7
:101D4000D5D11D4B1B78013B022B03D91B4B1B78B4
:101D5000022BCCD16C20C8E79809FF1FFC0FFF1F96
:101D60005C66FF1FFF3F0000141003406066FF1F0A
:101D70000C10034000100340D50BFF1F7211FF1F12
:101D8000B40003408C09FF1F680AFF1F490AFF1FA8
:101D900094000340460AFF1F470AFF1FF908FF1F70
:101DA0002209FF1F300DFF1F3409FF1FBC0BFF1F4F
:101DB000440AFF1F450AFF1F1C09FF1F2309FF1FBD
:101DC00010B502F00DF90022014B1A8010BDC0467B
:101DD0005866FF1F10B502F0EBF8A121054A8900F3
:101DE0009478054A61431268044B5218528C1A8049
:101DF00010BDC046300DFF1F3409FF1F5866FF1F7E
:101E000010B50D4B0D4A9978A1239B004B431268E6
:101E1000D218531DD97F0A4B1B88994209D2441C02
:101E200007D0C82805D0D2695B1A5A43054B5343E3
:101E3000C01802F05DF910BD300DFF1F3409FF1FFF
:101E40005866FF1F7102000070B5244D2B68002BEF
:101E500028D002F0E5F82B68D8402B680400002B4E
:101E600027D002F085F92B68D8401D4B1D4A997880
:101E7000A1239B004B431268D118D25C91239B0095
:101E8000002A20D0CA580132CA50174B17491B6884
:101E90000868834214D3D23B181A012A1AD0144B73
:101EA000186070BD02F0BCF8124B196802F0B8F966
:101EB000D3E702F05DF90F4B196802F0B1F9D4E7EE
:101EC0000D495B18E8E7CA500C4B1B68DB68E41847
:101ED000201AE4E7F530FF30E1E7C0461C08FF1F99
:101EE000300DFF1F3409FF1F9C09FF1F5C66FF1F99
:101EF000A009FF1F1808FF1F2DFF3F006466FF1F8A
:101F000070B504000D00282916D10300A433C2883F
:101F10001B889B1A0B4A9BB293420DD906006A3666
:101F200005223100653002F04BF9002804D1310060
:101F3000200002F0ADF870BD2900200002F038F951
:101F4000F9E7C046FE7F0000F8B50400012001F06B
:101F50006FFF02F04DF8174A174910600968030037
:101F60001648174E01601748776805680020AF4291
:101F700001D27068281A144D091928601348C162EB
:101F8000A421446A49032143416211490978002987
:101F900005D010490978022902D10F3B1360F8BD22
:101FA000012901D1083BF9E7032901D1053BF5E7F8
:101FB000033BF3E7E408FF1F28F00040340AFF1F4B
:101FC00028100040180AFF1F1C0AFF1F00F00040E5
:101FD0001C09FF1F4A0AFF1F70B580241025E40565
:101FE000A3682B43A36001F0EBFFA368AB43A3609E
:101FF00070BD0000F7B5160080221C001023D2052A
:102000000191916805000B43936000225A4BD73031
:102010001A6001F09DFF9D232A002F009B00EB58C2
:10202000CA3201210092FC37002B01D00021009A16
:10203000386801F07DFF2900009BCB311A784F4BA7
:10204000D3351A604B780A781B0213438A7812043E
:102050001A43CB781B061343494A1BBA13604B79CA
:102060000A791B0213438A7912041A43CB7931008F
:102070001B061343434A1BBA13606B782A781B0272
:102080001343AA7812041A43EB781B0613433E4A03
:102090001BBA1360019A330213433C4A13603C4B52
:1020A00022001B1B9C4603293DDCB3089A00130049
:1020B0005142B21A032A46D1354AE018511A8278A1
:1020C0004078120400020243E05C043302430A60D9
:1020D0000022FF2B4BDDF0222E4B12011A600F2243
:1020E0002D4B1A602D4A1368002BFCD00023224A86
:1020F00027491360091B321D0B191B68043A180A83
:1021000023706070180C1B0EA070E3700434002A5A
:10211000F2DC802210213B68D20501333B609368DA
:102120008B439360F7BD6346D578981893782D0656
:102130001B042B43157804392B43557804322D02A8
:102140002B430360AFE7022A0AD1114AE05C511A1F
:10215000E2185278120202430A6004339BB2B7E7D6
:10216000012AB5D10A4A521AE15C1160F5E7084923
:1021700059180A600433ACE7000004403C000440F6
:102180003800044034000440300004400C00044097
:102190000001044004000440100004401400044006
:1021A000F7B5150080221C001023D205009191681C
:1021B00007000B4393600023654AD730136001F09A
:1021C000C7FE9D233E009B00F9583B00CA363200F3
:1021D000FC33002900D07FE0586801F0A9FE3900E7
:1021E00032785C4BCB311A604B780A781B02134370
:1021F0008A78AC4612041A43CB78281D1B06134379
:10220000554A1BBA13604B790A791B0213438A792A
:1022100012041A43CB791B061343504A1BBA1360AE
:102220004B7A0A7A1B0213438A7A12041A43CB7A36
:1022300021001B0613434A4A1BBA1360009A2B0263
:102240001343484A13602200474B1B1B0093009B1B
:10225000CE785B1801938B7836061B0433430E78D7
:10226000043833434E78043136023343019E3360E1
:102270000328ECDC0321A808431C9B0029408000B4
:1022800003292BD13849E5185E18A9786D78E35CED
:1022900009042D022943194331600300083300214A
:1022A000FF2B2DDD314B324919600F21314B196065
:1022B000012327490B60304B19680029FCD0062107
:1022C0001B680B40042B20D080220020D20593688D
:1022D0000A318B439360FEBD01217DE7022908D1BD
:1022E00021495D18E1184978E35C09021943296026
:1022F000D3E70129D3D11C495918E35C0B60CCE723
:102300001948181801600433CAE7002310490B600C
:102310006346002B0CDC3B00FC335A681021013271
:102320005A608022D205936801208B439360D2E7E4
:10233000009B9B181B68190A13705170190C1B0E17
:10234000D37004235B4291709C440432E0E7C046A2
:10235000000004403C0004403800044034000440C5
:10236000300004400C00044000010440040004401C
:10237000080F0000100004401400044070B5061E51
:1023800019D00222614B9B799343012B13D1604BEF
:102390001A78FF2A0FD15A78FF2A0CD19A78FF2A8F
:1023A00009D1DA78FF2A06D11A79FF2A03D15B799D
:1023B000FF2B00D1A7E0574B0C201A78012A08D038
:1023C0000022554D1A702B781A00093A042A01D8B8
:1023D000212070BD5A1F012AFAD94C4CA07B042839
:1023E00000D990E0A279032A00D98CE0821E012A4C
:1023F00003D862881F2A00D885E0002E61D0012E04
:1024000000D080E0A288012AE2D0002B0AD1013856
:10241000032803D801F066FC151D19151F202E7026
:1024200001F0D6FE2B785A1E032A16D800253B4B06
:102430001D602823237501F01BFEA8422ED0A58025
:10244000C6E7022320202B70EAE7042322202B700A
:10245000E6E7032321202B70E2E7073B012BB7D8E7
:102460002F4B1B68DB6A9B06B2D52E4B1A78002ACD
:10247000AED1A27B911E012901D9002AA8D1022246
:1024800080211A702823284D89012878237501F0AE
:10249000CFFE80212878890101F05AFC0123A38016
:1024A000224B1B78002B0AD0FA228021204B92006D
:1024B0001B8809025A431C4B187801F0F9FC0020D4
:1024C00087E701F035FC2B78A680073B012B06D966
:1024D00018482E7001F014FE1E2001F079FE114BF9
:1024E000114C1A78002A06D0802100222078890118
:1024F0001A7001F09DFE01F083FE80212078090210
:1025000001F096FEDBE7122063E7C046A60BFF1F33
:102510006B09FF1F1A09FF1F1C09FF1F4809FF1F36
:102520006466FF1F2309FF1F1B09FF1F2109FF1FEF
:102530002C09FF1F0010004010B5002901D001F048
:102540008FFC10BDF7B5604B01919978A1239B00DA
:102550004B435E4A060014681022E418D6235B0041
:10256000E0583623FF33E35C00279343222B41D10D
:10257000574B0F3A1A600760012501F0D1FB019B10
:102580001880E8235B00E35C002B01D0B34258DDE8
:102590000023504FFB70AD33FF33E3581A68002A15
:1025A00003D09B88DB439B071DD03823FF33E35CBC
:1025B000002B18D09B235B00E35C002B13D1D1339D
:1025C000FF33E35CB3420EDAA4235B00E15AE01868
:1025D000090A023101F0DCFD23000122FE33013E35
:1025E00001351A87FA70E8235B00E35C002B2AD0E0
:1025F000A8B2FEBD03683D00002BBED08188043028
:10260000090A023101F0C4FDD6235B00E3581F60C4
:10261000B2E72300B133BA00FF33985801378188FD
:102620000430090A023101F0B3FDE8235B00E35CEA
:10263000BB42EEDCE822F61AED1800235200A35448
:10264000A6E70027F1E7200001F0C2FB00281FD019
:10265000002E1DDD7319882647190193B60020004E
:1026600001F016FC5A30800020184068013581883E
:102670000430090A023101F08BFD200001F098FBC3
:10268000A3590133A351BD4202D0019B9D42E6D123
:10269000114BE35C002BABD095239B00E35C002B3C
:1026A000A6D00E4BE15A0029A2D00D4AA35C994254
:1026B00002D90133A3549BE700231A212000A3541D
:1026C00001F026FB94E7C046300DFF1F3409FF1FC1
:1026D00000140340E010FF1F5A02000072020000C5
:1026E0005E020000F8B51D4B1D4F1A78002A10D16C
:1026F000BA7B002A02D101321A7003E0032AFAD011
:10270000022AF8D001F0B4FC00220120154B1A7007
:10271000F8BD154B154D1C68154B9E7801232B7089
:102720002878C0B200F0DEFCBB7B002B0BD101F09F
:102730006FFCA1239B007343E41883239B00E418E0
:1027400023782B70E4E7032B02D101F081FCF0E742
:102750000020022BDCD101F093FBEAE71C09FF1FEC
:10276000A60BFF1F2309FF1F3409FF1F490AFF1F84
:10277000300DFF1FF0B587B00EAD2F780FAD2D785F
:102780000593AC46634614000E4D0CAA12782E78C1
:1027900003930D9B009201932200059B029701F089
:1027A00097FC2E70012C01D0042C08D18022064900
:1027B0008B889343054A1278D20113438B8007B06C
:1027C000F0BDC0461C09FF1F6C11FF1F7809FF1FD9
:1027D0000B001B3B70B504003020E02B0DD813001C
:1027E000E025493BFF3B9BB2ED00AB4205D8034BD4
:1027F000200019825A8201F0E3FA70BD8410FF1F95
:1028000010B501F015FC054B00205B68052B04D9C1
:10281000034A5268D20200D4980810BD001000404C
:10282000FCE100E070B501F083FA0D4B1B68FC334E
:10283000DC691D6AFFF7E4FF6419844204D2094B86
:1028400001241B68002B07D004220024064B1A70B9
:10285000064A93690133936101F0D2FC200070BDF8
:102860006466FF1F9809FF1F2309FF1FFC0FFF1F4E
:1028700070B50C4D2B68FC335C6A01F059FAFFF718
:10288000BFFF2B680025FC339B6AE318834204D208
:10289000054B1B68AB4200D1051B01F0B1FC2800C1
:1028A00070BDC0466466FF1F9809FF1FD722044B06
:1028B00092009B5810B5002B00D0984710BDC04621
:1028C0000000FF1FF0B587B001F096F9FFF7EEFFAB
:1028D000CA4BCB4C04931B78022B45D1C94B1B68C8
:1028E000186A01F0A5FAC84BC84A1A60C84BC94A11
:1028F0001A60A022C84B52001A60049B187801F09D
:10290000BFFBC649C64801F08BFAC649C64801F06C
:1029100087FA1022C54BFF201A60802252031A60EA
:10292000802292031A60802212041A6001F008FCCF
:10293000012001F025FCFA20400001F0C1FB5820E5
:1029400001F026FABA4801F0C3FA012001F018FAA2
:10295000072001F07DFC2268B64B1A4084235B00FF
:102960001343236007B0F0BD01F0FAF9B24E0290B4
:10297000322001F05DFA33681B0629D43C2001F0B7
:1029800057FA0F2001F054FA9C4B1B78012B00D111
:102990001EE180223368A94D134200D0A7E02B68C6
:1029A000032013432B6001F043FA01F0D9F9029B95
:1029B0000299C31A5A1E814200D81A00A04B1A600D
:1029C000904B19681E2353439E4A9B18CB618AE79C
:1029D00001F0C6F980239C4ADB02116803900B4387
:1029E00013602268934B994F1A40282313432360A6
:1029F000032001F01DFA03203D6801F019FA3B683D
:102A00000320DB03DB0B009301F012FA3B68ED03BC
:102A1000DB03ED0BDB0B8E4A0193AB18C22B30D8D6
:102A2000009B9B18C22B2CD8019B9B18C22B28D82B
:102A3000009B2A009D4200D21A00009B9D4200D9B3
:102A40001D00019B934200D21300019A954200D9C8
:102A500015005B1B122B14D80C22336814209343EF
:102A6000336033687B4A1340336001F0E1F9082199
:102A70003B682268DB038A432260774ADB0B1360E2
:102A80007FE7032001F0D4F93B68DB03DB0B059300
:102A900001F066F9039B0399C21A531E814200D8C4
:102AA00013006E4A93421BD9FF23356869492D0AEA
:102AB0001D4032686B1C1B060A401B0C134333601D
:102AC0000C23326800209A43083B1343336001F023
:102AD000B7FB6348634BA840984206DCFEF732FF21
:102AE000019B009D0093059B95E75F48F6E7002357
:102AF0005E4F554A3B6080231168DB020B43136035
:102B000080222B68032013432B6001F091F93B686E
:102B1000052601333B6080232A685B0213432B6048
:102B20002268444B03201A40514B1343236001F0A9
:102B30007FF90821454B1A682368D2038B43236031
:102B4000454B023900931B68D20B4B439A420CD879
:102B50009B1A3B2B0BD8236846490B4023602B68FC
:102B60000B402B60444B1A601FE7D31AF1E7013E7C
:102B7000F6B2002ED4D123683E4A134023602B685E
:102B800013402B603B68042B07D9BFF34F8F3B4B9F
:102B90003B4ADA60BFF34F8FFEE780222B680320A9
:102BA00093432B6001F044F92268224B03201A4022
:102BB00028231343236001F03BF9244B009A1B6840
:102BC000DB03DB0B1360082223689343236097E742
:102BD00007222C4D2B681340012B02D1002001F05D
:102BE0004FFAAB68284A02201340AB6001F020F98D
:102BF0008023AA685B001343AB60D6E64A0AFF1F36
:102C00005CF000406466FF1F000003400180063D49
:102C1000BC00034034080000A4000340710200001F
:102C200014100040FFFF3F002810004000E100E0CA
:102C30003075000000FEFEFFC4F0004044F000408C
:102C40004C66FF1F7206000040F0004064F0004038
:102C500091FCFFFFFF00FFFF5466FF1FE30C000025
:102C6000E88000005F361E0060361E00B844FF1F7B
:102C700028000100FFFFFEFF5066FF1F00ED00E08F
:102C80000400FA053CF00040FFFEFFFF694E336888
:102C900088331B6883F3088801F09AF900F014FC6C
:102CA000654B664A1B68934207D0002001F0C8FAC2
:102CB0000221634A13688B431360FFF703FE614BE5
:102CC000614C1878C0B201F0EBF80023A360023326
:102CD000A3605E4B0120236001F0AAF80323A360E8
:102CE00001F03EF8040001F0A3F9050001F038F806
:102CF000574B186001F0F4F9564B1968621A531ECD
:102D0000A14200D213008022D203934201D39B023E
:102D10009B0A3268D16AC90700D478E04E491C0C7E
:102D200009689BB24C4359432402090A64180327DB
:102D30004A49FC3293680A6849489B1A494A4A4EF4
:102D400012684A499B18414A34609A183B400193E3
:102D5000036892089C46019B0A6063440360042B4D
:102D600003D901323B400A6003600B684049E41814
:102D7000200001F055FA3F4F3D493B68C3183B60C6
:102D80002000019301F09CF83B4C2068081838495A
:102D90002060884205D9019B01333B6001F090F827
:102DA000216001F02DF9354B1B78002B0ED001F07E
:102DB0003FF93168324B4A1B1B6812189A4233D2D2
:102DC000591A4919091A2F4801F02AF82E4C237A6A
:102DD000002B0FD001F02CF93168E3684A1B121860
:102DE000934224D9591A4919091A284801F018F8A8
:102DF00000232372264B83F3088800F0A1FF0220F2
:102E000001F0E6F9002001F01BFA01F051F9DC01B4
:102E100099000234641A5900641A09214B43803323
:102E2000CB40A408E41882E7FA218900CBE71949CE
:102E3000DBE7C0466466FF1F0C0AFF1FB641210393
:102E400010000040490AFF1F14100040C409000090
:102E5000100AFF1F340AFF1F380AFF1F200AFF1F36
:102E6000280AFF1F1C0AFF1F4866FF1F240AFF1FB6
:102E7000710200006008FF1F2C0AFF1F1C09FF1FC2
:102E8000E408FF1F00100040740BFF1F3C100040BF
:102E900000000020DC050000A022054B92009B589A
:102EA00010B5002B01D0984710BD00F0A1FFFBE743
:102EB0000000FF1FA122054B92009B5810B5002B6C
:102EC00001D0984710BD00F093FFFBE70000FF1F03
:102ED000A222054B92009B5810B5002B01D09847B9
:102EE00010BD00F085FFFBE70000FF1FA322054B8C
:102EF00092009B5810B5002B01D0984710BD00F0F0
:102F000077FFFBE70000FF1FA422054B92009B58B0
:102F100010B5002B01D0984710BD00F069FFFBE70A
:102F20000000FF1F70B501F083F8514B18600420BA
:102F300001F04EF900F054FF0400C30702D401F081
:102F40002FF870BD00224B4B1A604B4B187801389C
:102F500004282CD800F0C6FE03231B1F27002000E6
:102F600000F0FEFF0128ECD0444C2378042B71D1F3
:102F700001F096F8002806D000F0D2FF582000F0AB
:102F800007FF02232370032001F022F9D9E7200074
:102F900000F03EFFE6E7200000F0D2FFE2E720006D
:102FA00001F04EF8DEE7200000F04AFFDAE701F01A
:102FB0001FF90500012808D1314B1B78053B012B77
:102FC00003D82000FFF768FFCEE72C4B1B78022BBD
:102FD00001D0052B20D1022D28D12A4B9B7BAB435E
:102FE0001CD12000FFF766FF254B18780128BBD1C4
:102FF0006405B9D4234925224B7B034205D1233AEA
:1030000013405A42534126331A000B7D9342ABD9E9
:10301000322001F08DF8A7E7022D07D1184B1B785D
:10302000052B11D12000FFF753FFDDE7012D0BD158
:10303000012B03D12000FFF759FF95E7062B03D1A1
:103040002000FFF761FF8FE7200000F0D1FE022D86
:103050008AD1C9E7032B04D10B4B987C01F000F80F
:1030600091E7072B8FD1094B987B01F079F88AE71C
:103070009C09FF1F9809FF1F9009FF1F2309FF1FCD
:103080001C09FF1FA60BFF1FBC0BFF1FD40BFF1F4C
:10309000FA210A4B0A4A49001A640A4A5A500A4A53
:1030A00004395A50094A08319A64094A5A50094A5F
:1030B0005C315A50084ADA667047C0460000FF1F6C
:1030C0007527FF1F7128FF1F2528FF1F7D23FF1F66
:1030D000E526FF1F011EFF1FD51DFF1F10B500F0C5
:1030E000E9FD10BD8023F7B59C46264B264F019382
:1030F0002649274A274D284C284B02281AD16046DA
:1031000038600868264E3040802636033043086019
:1031100001990978002909D11660224A2A60224AB9
:103120002260E02219689143A03A1BE08021C90285
:103130001160F2E766463E600F68194E3E408027F8
:10314000FF023E430E600199097800290DD11760F6
:1031500001280ED1154A2A60154A2260E02219681A
:103160009143C03A0A431A60F7BD80218902116079
:10317000EEE7E0210F4A02432A600F4A22601A68F4
:103180008A43F0E74B0AFF1FE0000340D8000340EA
:103190009000034000000340500003404000034003
:1031A000FFFFE3FF0280063D804508220180063DC7
:1031B000806608220080069880550822F8B51E4BCC
:1031C00080261A68002014003440324232D11A6836
:1031D0001A4F32431A6001223B68063093433B602A
:1031E00000F026FE0122164D2B681E432E603B6820
:1031F0000A2613433B608027BF00124B1B683B42EB
:1032000011D1013EF6B2FF2E09D17E220E4B1C6871
:103210002B68E40B1440934323432B6005E0082004
:1032200000F006FEE9E7002EEFD180222B6860084F
:1032300093432B60F8BDC046C4F000405CF00040F2
:1032400018F0004068F0004060F0004010B500F059
:10325000A7FF01215820034A00F08AFDFFF7AEFFC7
:1032600010BDC046600AFF1F10B578220021034838
:1032700000F06EFF00F04CFF002010BD6C69FF1FD6
:1032800070B5040000F054FD00230C200B4A01002F
:1032900059438D18515C00290DD0A14208D101235A
:1032A00000246B7000F07CFD00F0AAFF200070BDD0
:1032B00001330A2BEBD11224F6E7C0466C69FF1FDD
:1032C00070B5040000F034FD002319001D000D4A04
:1032D0001078002806D0A0420CD1557001310C3274
:1032E0000A29F5D1002B0AD100F012FF00F088FF67
:1032F000002070BD5078461EB0411B18EEE700F06C
:103300004FFDF3E76C69FF1FF7B504000C200023A5
:1033100084460E4D019267465F43E85D7E19A042E8
:1033200012D000280BD10A4B9C4662461B7808330A
:103330001370019B70707C557160B360FEBD0133EA
:103340000A2BE8D10320F9E70720F7E76C69FF1F94
:103350006869FF1F8021F8B5464BC9051B68C12469
:103360008B60454BFF261A68012313434B61434B87
:10337000A4001A68424B40201A60424B1A68424B24
:103380001A60424B1A59B2431A51C52292009D58F5
:10339000B5432843802598509F583D48ED0107408C
:1033A0003D439D509D5880272D022D0A2943995059
:1033B00080211A59090202400A431A5104341A5949
:1033C000344D3F042A403A4380271A511A593F0688
:1033D0001202120A3A431A5108341A5902400A4397
:1033E0001A51C32292009D58B5432C0080252C43CE
:1033F0009C509D582C0004400C439C509D58254CDB
:1034000025408024240425439D509C588025240277
:10341000240A3C439C50C424A4001A59B2432A43B2
:103420001A511A591202120A17431F5108341A5915
:10343000B24315431D5100251A5902400A431A513F
:1034400004341A59024011431951134C134B1B7881
:10345000DB08AB4201DC0020F8BD2378002B06D04E
:10346000A368002B00D0984701350C34EEE71220FA
:10347000F2E7C0465045FF1F4C45FF1FB0F000402B
:103480006469FF1FB4F000406069FF1F00E100E0C5
:10349000FF00FFFFFFFF00FF6C69FF1F6869FF1F50
:1034A000030010B51F2809D8072200201340072465
:1034B00004490A78A24313430B7010BD0023062071
:1034C000F5E7C0466869FF1F034A044913680020F6
:1034D0000B4013607047C0461CF00040FFFFC1FF67
:1034E000054B06491B780A6805485B0702401B0B21
:1034F000134300200B6070476869FF1F1CF00040F9
:10350000FFFFC1FF70B50C25FFF7EAFF0A4B1C78DF
:103510000A4BE4086543ED18002C01D1200070BD72
:103520002B78002B06D06B68002B00D09847013C0D
:103530000C3DF1E71220F2E76869FF1F6069FF1F89
:1035400007B50422074801A900F034F9019B0133B3
:1035500005D18023044ADB0411680B43136000206B
:103560000EBDC0461C18001114F00040F0B5050057
:103570002026184B87B00493049B002B03D1112401
:10358000200007B0F0BD002102220B000191009144
:10359000052000F0EDFC02230F490A681A42FCD115
:1035A0000596059C631E0593002CFAD10B4A1368FF
:1035B000002BFCDA0F276F440121380000F090FC4B
:1035C0003B782B42DCD0052000F032FC049B013B11
:1035D0000493D1E7FFFFFF0790C8004000C80040F8
:1035E00007B500F0A5FB80220821D205936A01915E
:1035F000002B01D10739916202210C4A1160019917
:10360000481E01900029FAD1033111600531019162
:103610000199481E01900029FAD11160002B02D1B6
:103620008022D205936200F0EBFD07BD00C0004090
:10363000F0B52D4C89B02378002B4FD1FEF762F9FD
:1036400002232A4F03903A681A42FCD120230693A2
:10365000069B5A1E0692002BFAD1254E3368002B8A
:10366000FCDA0120FFF782FF011E02D0112009B011
:10367000F0BD030003220190009005AD9F2000F0F3
:1036800077FC0321280000F02BFC02233A681A4241
:10369000FCD120230793079B5A1E0792002BFAD1D7
:1036A0003368002BFCDA0120FFF760FF0028DDD132
:1036B0000398FEF73BF9AA786B7811041B020B43C1
:1036C00029780B4363601300113B0A49052B07D887
:1036D00001239340A3600B60012323700020C6E701
:1036E00080231B03F6E7C0463845FF1F90C8004003
:1036F00000C800409808FF1F1E4B30B55A68187864
:103700001D4B85B0D31859424B4101210093002332
:1037100000F036FC194B1A4A02259A6300221A65FA
:1037200010325A658022C4219D65164B1648D2027C
:10373000DA6789004258154B80241A4080231B0405
:1037400013434350642341200393E40500F078F9C8
:10375000402000F075F96562039D6B1E0393002DF8
:10376000FAD103236362FFF73BFFA562FFF760FF17
:1037700005B030BD4445FF1F95FFFEF700C800406F
:10378000050001FF04E100E000E100E0FFFF00FFB1
:1037900010B5064B18705960FFF7AEFF00211320DB
:1037A000034AFFF7B1FD002010BDC0464445FF1F8E
:1037B000F936FF1FF0B5040085B003920291FEF7C1
:1037C000A1F8882263035B0B52051A438023DB05B3
:1037D0009D6A8023274F0092BA68002601901B0340
:1037E0009A420CD9F82326001B041E401C4206D026
:1037F0008022214B52025E6219680A431A60002D32
:103800000BD100F095FA02221C4B1A608023DB05D5
:103810005A62013A9A6200F0F3FC0023039A934241
:1038200020D1002D0AD100F083FA144B03221D6031
:103830008023DB055A629D6200F0E2FC8023BA68B7
:103840001B039A4208D9002E06D000220A4B0C49CD
:103850005A621A680A401A600198FEF767F8002059
:1038600005B0F0BD009A0299D2181278CA540133FB
:10387000D4E7C0463845FF1F00C8004000C00040E4
:10388000FFFFFEFFF0B587B0029103920400FEF740
:1038900039F8019000F04CFA802302250122234ED2
:1038A000DB0535605D629A6200F0AAFC204F3B6840
:1038B0002B42FCD120230493049B5A1E0492002B1C
:1038C000FAD11C4D2B68002BFCDA0120FFF74EFECD
:1038D000002802D0112007B0F0BD2000039A029901
:1038E00000F07EFC022304003A681A42FCD1202337
:1038F0000593059B5A1E0592002BFAD12B68002BCD
:10390000FCDA0120FFF732FE051EE3D100F010FAC9
:1039100080230322DB0535605A629D6200F070FC53
:103920000198FEF703F8E0B2D5E7C04600C00040BA
:1039300090C8004000C80040F0B5802687B0040061
:10394000FDF7E0FFF605B36A02250393029000F04D
:10395000EFF90123244F3D607562B36200F050FC23
:10396000224E33682B42FCD120230493049B5A1E21
:103970000492002BFAD11E4D2B68002BFCDA01209B
:10398000FFF7F4FD002802D0112007B0F0BD2000A1
:1039900000F0B6FA0223019032681A42FCD12023CB
:1039A0000593059B5A1E0592002BFAD12B68002B1C
:1039B000FCDA0320FFF7DAFD041EE5D100F0B8F9C8
:1039C00080230322DB053C605A629C6200F018FCF5
:1039D000039B002B01D1FFF703FE0298FDF7A6FF22
:1039E0006B461879D1E7C04600C0004090C800403F
:1039F00000C8004007B5000201910422000A01A995
:103A0000FFF740FF0EBD000073B5050005240B4A0B
:103A1000A3005B429B1819686B46DE1D300000F066
:103A200067FA022804D133782B55013CEFD276BDDA
:103A3000052CFCD00128FAD10230F8E71409001156
:103A40001F2807D8012380228340D20591680B43A9
:103A5000936070473F2808D8012380222038834094
:103A6000D20551690B435361F3E75F28F1D8012375
:103A7000802240388340D205116A0B431362E8E785
:103A80001F2807D8012280218240C9058B689343F3
:103A90008B6070473F2808D801228021203882405F
:103AA000C9054B6993434B61F3E75F28F1D80122C5
:103AB000802140388240C9050B6A93430B62E8E7D6
:103AC0001F2810D880230200DB05153A1968012A47
:103AD00006D820229143196019680A431A6070477A
:103AE00001228240F6E73F2811D880230200DB053F
:103AF000353AD968032A06D810229143D960D9688B
:103B00000A43DA60EBE7012220388240F5E75F28BC
:103B1000E5D842238022181A413B8340D205516ADE
:103B200099435162516A0B435362D8E710B50400C0
:103B3000012813D1A022184992050B685B015B098B
:103B400013430B60154B164A19681140154A0A4376
:103B50001A60402219680A431A6010BD0028FCD17F
:103B600001000A2000F014FA21000B2000F010FAE6
:103B7000C0220A4B920019680A4340211A601A6851
:103B80008A431A60B022044912060B685B015B0984
:103B900013430B60E1E7C04614F000401CF0004006
:103BA0007F00FEFF80FD010072B6074A13680133F3
:103BB00013600422054B1A600023054A136080221B
:103BC000D2055360FEE7C0467808FF1FC0F00040F2
:103BD000C4F00040044B054A1A60054B1A600022ED
:103BE000044B1A607047C046140AFF1F841E000071
:103BF000380AFF1FC4F000400023034A1360034A41
:103C00001360034A1360704754F0004040F10040D5
:103C100044F10040002310B5184C8AB00093019382
:103C20002378012B27D06946012000F079FA00287B
:103C300017D1009B12490293019B06AA0393114BD3
:103C400002A81B680493104B1B68059300F0B8F999
:103C500010220E4906A800F0B3FA002804D1FF2371
:103C6000237000200AB010BD0123094A074902A8A9
:103C7000237000F0A5F90120F4E7C0466866FF1F35
:103C800010290011082900110C2900112029001108
:103C90006C66FF1F13B501246946012000F040FA4D
:103CA000034B00940193FFF7B5FF200016BDC046FB
:103CB000BB0B000010B5FFF79FFFFFF7EBFF0028DD
:103CC00002D0024B984710BDFEE7C046E1A20000BB
:103CD00002B4714649084900095649008E4402BCA5
:103CE0007047C04602B4714649084900095C490062
:103CF0008E4402BC7047C04603B471464908400078
:103D00004900095A49008E4403BC70470000000076
:103D100001B40248844601BC604700BF53B90000AB
:103D200001B40248844601BC604700BFCD0C0100CD
:103D300001B40248844601BC604700BF75A9000079
:103D400001B40248844601BC604700BF7997000077
:103D500001B40248844601BC604700BF0D52010017
:103D600001B40248844601BC604700BF156B0100E6
:103D700001B40248844601BC604700BF01670100EE
:103D800001B40248844601BC604700BFE51201004F
:103D900001B40248844601BC604700BF79120100AB
:103DA00001B40248844601BC604700BF21A900005D
:103DB00001B40248844601BC604700BF5976010047
:103DC00001B40248844601BC604700BF116E000088
:103DD00001B40248844601BC604700BF71B00000D6
:103DE00001B40248844601BC604700BFBD0B01001E
:103DF00001B40248844601BC604700BFE9170100D6
:103E000001B40248844601BC604700BFF9A6000027
:103E100001B40248844601BC604700BF0934010078
:103E200001B40248844601BC604700BF2D6C01000C
:103E300001B40248844601BC604700BF018900000C
:103E400001B40248844601BC604700BFF935010057
:103E500001B40248844601BC604700BFE94C010040
:103E600001B40248844601BC604700BFE9D40000A9
:103E700001B40248844601BC604700BF9DB60011F2
:103E800001B40248844601BC604700BF19FA000033
:103E900001B40248844601BC604700BFD9B00000AD
:103EA00001B40248844601BC604700BF8914010088
:103EB00001B40248844601BC604700BF8B52010038
:103EC00001B40248844601BC604700BF090E0000EF
:103ED00001B40248844601BC604700BF8D11010057
:103EE00001B40248844601BC604700BF3D71010037
:103EF00001B40248844601BC604700BF8D38001100
:103F000001B40248844601BC604700BFA96F0100AC
:103F100001B40248844601BC604700BFE9270000A5
:103F200001B40248844601BC604700BF6DF6000042
:103F300001B40248844601BC604700BF2144000030
:103F400001B40248844601BC604700BF053401004B
:103F500001B40248844601BC604700BF89440000A8
:103F600001B40248844601BC604700BF013401002F
:103F700001B40248844601BC604700BF496D01009E
:103F800001B40248844601BC604700BFC56D010012
:103F900001B40248844601BC604700BF8DA20011F5
:103FA00001B40248844601BC604700BFDD0A01003D
:103FB00001B40248844601BC604700BFF9ED00002F
:103FC00001B40248844601BC604700BFDD3F0000E9
:103FD00001B40248844601BC604700BFC9A9000083
:103FE00001B40248844601BC604700BF8D820000D6
:103FF00001B40248844601BC604700BFBD5C0100BB
:1040000001B40248844601BC604700BFD5440100AA
:1040100001B40248844601BC604700BFE9F60000D5
:1040200001B40248844601BC604700BFE90B0100AF
:1040300001B40248844601BC604700BFC95C01006E
:1040400001B40248844601BC604700BFF535010059
:1040500001B40248844601BC604700BF75F8000007
:1040600001B40248844601BC604700BF4DF900001E
:1040700001B40248844601BC604700BFA9D80000D3
:1040800001B40248844601BC604700BFEDA50000B2
:1040900001B40248844601BC604700BF85C10000EE
:1040A00001B40248844601BC604700BF01D700004C
:1040B00001B40248844601BC604700BF855201003C
:1040C00001B40248844601BC604700BF851201006C
:1040D00001B40248844601BC604700BF9D6A0000ED
:1040E00001B40248844601BC604700BFC1660100BC
:1040F00001B40248844601BC604700BF8937010013
:1041000001B40248844601BC604700BFC1A500005D
:1041100001B40248844601BC604700BFADAE000058
:1041200001B40248844601BC604700BFE1AC000016
:1041300001B40248844601BC604700BF61370100FA
:1041400001B40248844601BC604700BFED6B01002A
:1041500001B40248844601BC604700BFB70E0000AE
:1041600001B40248844601BC604700BFC1F70000AB
:1041700001B40248844601BC604700BF6D0B0100DA
:1041800001B40248844601BC604700BF69110100C8
:1041900001B40248844601BC604700BFC11501005C
:1041A00001B40248844601BC604700BFED680100CD
:1041B00001B40248844601BC604700BF51B800000A
:1041C00001B40248844601BC604700BFCD4C0100E9
:1041D00001B40248844601BC604700BF19070100D2
:1041E00001B40248844601BC604700BF95730100DA
:1041F00001B40248844601BC604700BFDD0C0100E9
:1042000001B40248844601BC604700BF9DA900007C
:1042100001B40248844601BC604700BFA1AF000062
:1042200001B40248844601BC604700BF090E00008B
:1042300001B40248844601BC604700BFB35201008C
:1042400001B40248844601BC604700BF016C010014
:1042500001B40248844601BC604700BFF90D01006B
:1042600002000000EABF001101000000A0BD001123
:1042700002000000E6BF001101000000A042FF1F85
:1042800002000000A8BD001101000000A863FF1F8C
:1042900002000000E4BF0011030000001C63FF1FC8
:1042A0001200000002000000EABF0011010000003F
:1042B000E8BD001102000000E6BF0011010000008F
:1042C000E5BD001102000000F2BD00110300000076
:1042D0005763FF1F02000000E4BF0011030000004D
:1042E0006C63FF1F02000000E6BF00110100000028
:1042F000E4BD001102000000F0BD00110300000049
:104300002D63FF1F02000000E4BF00110300000046
:104310004E63FF1F02000000EABF00110100000011
:1043200028BE001102000000E6BF001101000000DD
:10433000E943FF1F020000003ABE00110100000027
:1043400023BE001102000000E6BF001101000000C2
:10435000E843FF1F0200000038BE0011010000000A
:104360007463FF1F02000000E6BF0011010000009F
:10437000E743FF1F0200000036BE001101000000ED
:1043800013BE001102000000E6BF00110100000092
:10439000E643FF1F0200000034BE001101000000D0
:1043A0000EBE001102000000E6BF00110100000077
:1043B000E543FF1F0200000032BE001101000000B3
:1043C00009BE001102000000E6BF0011010000005C
:1043D000E443FF1F0200000030BE00110100000096
:1043E00004BE00110202020202020000F54B00119D
:1043F000BB4B00117CBE0011900118001800FFFF9C
:104400000701020304050602010600000000000087
:10441000000000000000000000000000000000009C
:10442000000000000000030002000000EABF0011CD
:1044300001000000FCBE001102000000E6BF0011F8
:10444000010000009844FF1F0200000006BF001199
:1044500001000000A263FF1F02000000E4BF001182
:10446000030000001066FF1F02000000E6BF0011FD
:10447000010000009844FF1F0200000004BF00116B
:1044800001000000A463FF1F02000000E4BF001150
:10449000030000000866FF1F12A6A6A60000000089
:1044A0000001000000000111FFFF000050485936D4
:1044B0000000000000000000010000008DBE00119F
:1044C0000B000500F7000000B400002800280028B9
:1044D0003075A000A000A000A00000080008E001C6
:1044E000F00010001000100010001000100050002C
:1044F0005000500010001000D00700000000000025
:104500000F0001000500307507001000010081FF59
:1045100000000000FF000000657400116D720011C2
:10452000FD6F0011FFFF0100FF000000819E0011E0
:10453000FD9B0011159B0011000000000000000011
:1045400000000800040000003B0001085902E001DF
:1045500088212800FF00000002000000EABF0011CF
:1045600001000000B0C0001102000000E6BF001111
:1045700001000000D545FF1F02000000E2BF00114E
:1045800001000000246AFF1F02000000E6BF0011C6
:1045900001000000D445FF1F02000000E0BF001131
:1045A00001000000D245FF1F02000000E6BF00111D
:1045B00001000000D045FF1F02000000DEBF001117
:1045C00001000000C845FF1F1800180000009001FE
:1045D000020000030202000002000000EABF001116
:1045E00001000000C4C0001102000000E6BF00117D
:1045F000010000001846FF1F02000000DCBF001190
:10460000000000000000000002000000E4BF0011F4
:0A46100003000000446AFF1F20FFB2
:040000051FFF184180
:00000001FF
